:020000040000FA
:100000000004040000000000041A0000081A0000A8
:100010000C1A0000101A0000141A00000C1B00003B
:100020000C1B00000C1B0000181A00001C1A00001A
:10003000201A0000241A00000C1B0000281A0000DF
:100040002C1A0000301A0000341A0000381A000080
:100050003C1A0000401A0000441A0000481A000030
:100060000C1B00000C1B00004C1A0000501A000072
:10007000541A0000581A00005C1A00000C1B000003
:10008000601A0000641A00000C1B0000681A0000CF
:100090006C1A0000701A0000741A0000781A000030
:1000A0007C1A0000801A0000841A0000881A0000E0
:1000B0000C1B00000C1B00000C1B00008C1A000025
:1000C000901A0000941A0000981A00009C1A000070
:1000D000A01A0000A41A0000A81A0000AC1A000020
:1000E0000C1B00000C1B00000C1B0000B01A0000D1
:1000F000B41A00000C1B00000C1B0000B81A000012
:10010000BC1A00000C1B00000C1B00000C1B0000A4
:100110000C1B00000C1B00000C1B00000C1B000043
:10012000C01A00000C1B00000C1B0000C41A0000C9
:10013000C81A0000CC1A00000C1B00000C1B0000A9
:100140000C1B00000C1B0000D01A00000C1B000050
:100150000C1B00000C1B00000C1B0000D41A00003C
:100160000C1B00000C1B00000C1B0000D81A000028
:10017000DC1A0000E01A0000E41A0000E81A00008F
:10018000EC1A0000F01A0000F41A0000F81A00003F
:10019000FC1A0000001B0000041B0000081B0000EC
:1001A0000C1B00000C1B00000C1B00000C1B0000B3
:1001B0000C1B00000C1B00000C1B00000C1B0000A3
:1001C0000C1B00000C1B00000C1B00000C1B000093
:1001D0000C1B00000C1B00000C1B00000C1B000083
:1001E0000C1B00000C1B00000C1B00000C1B000073
:1001F0000C1B00000C1B00000C1B00000C1B000063
:10020000FFFFFF00FFFFFF00C8040000C80400005C
:10021000C8040000C8040000C8040000C8040000AE
:10022000C8040000C8040000C8040000C80400009E
:10023000C8040000C8040000C8040000C80400008E
:10024000C8040000C8040000C8040000C80400007E
:10025000C8040000C8040000C8040000C80400006E
:10026000C8040000C8040000C8040000C80400005E
:10027000C8040000C8040000C8040000C80400004E
:10028000C8040000C8040000C8040000C80400003E
:10029000C8040000C8040000C8040000C80400002E
:1002A000C8040000C8040000C8040000C80400001E
:1002B000C8040000C8040000C8040000C80400000E
:1002C000C8040000C8040000C8040000C8040000FE
:1002D000C8040000C8040000C8040000C8040000EE
:1002E000C8040000C8040000C8040000C8040000DE
:1002F000C8040000C8040000C8040000C8040000CE
:10030000C8040000C8040000C8040000C8040000BD
:10031000C8040000C8040000C8040000C8040000AD
:10032000C8040000C8040000C8040000C80400009D
:10033000C8040000C8040000C8040000C80400008D
:10034000C8040000C8040000C8040000C80400007D
:10035000C8040000C8040000C8040000C80400006D
:10036000C8040000C8040000C8040000C80400005D
:10037000C8040000C8040000C8040000C80400004D
:10038000C8040000C8040000C8040000C80400003D
:10039000C8040000C8040000C8040000C80400002D
:1003A000C8040000C8040000C8040000C80400001D
:1003B000C8040000C8040000C8040000C80400000D
:1003C000C8040000C8040000C8040000C8040000FD
:1003D000C8040000C8040000C8040000C8040000ED
:1003E000C8040000C8040000C8040000C8040000DD
:1003F000C8040000C8040000C8040000C8040000CD
:100800000FA220000E7F24000E01880000000000CF
:10081000000020000000E000020032000001200083
:1008200020028800140007005B0007000000E000C1
:1008300003003A0080682100010020000200370018
:100840000000200001002000810F70000100320034
:1008500014000700000020000000E0000200320049
:100860000000020000000000DC1402000000000094
:100870000040DA000000FE004440A90040112000C2
:100880000000E0000300320000002000A00188000A
:100890004440A800000006008A1F78008B1F7800E3
:1008A0000000060091018800800478000000EB0041
:1008B0001A003700E284440032A0B4009905BA005F
:1008C000E284440032A0B4009906BA00E2844400F5
:1008D00032A0B4000006EB00476FDE00FD07B20057
:1008E000636CE10003003A00EBFF07000000EB003F
:1008F0000A003700606CE10004003A00005DEB0084
:100900008B05E900FDFF3E00040037006168E1004F
:10091000010032000086EB000B00070019C7BA0087
:100920001905BA000E04E00003003A000A00E000D6
:10093000E0FF3A0000000600FE07B2009E018800BA
:100940008A047800F5FF3700395DBA008B05E900AD
:100950000C003200295DBA008B05E9000800320066
:100960000C00E00003003A00E284440032A0B4002E
:10097000F5FF370019DDBA008B05E900FAFF3A00F0
:100980008904E800E184440032A0B40000000600BD
:100990000040DA000000FE00000005008001780041
:1009A00002003700815978000201E9000200E000EE
:1009B000FCFF3A00000006001201000000020000E7
:1009C0000000000000080000D80400003C00000007
:1009D0000001000001020000000100000902000007
:1009E000290000000101000000C0000032090000E1
:1009F00004000000000200000300000000000000EE
:100A0000092100001101000000010000221D00006A
:100A10000007000005810000034000000001000005
:100A20000705000001030000400000000100000075
:100A30000403000009040000340300004D0000001E
:100A40006900000063000000720000006F000000F9
:100A500063000000680000006900000070000000F2
:100A6000200000005400000065000000630000004A
:100A7000680000006E0000006F0000006C000000C5
:100A80006F000000670000007900000020000000F7
:100A9000490000006E000000630000002E0000000E
:100AA0002603000055000000530000004200000033
:100AB0002000000048000000490000004400000041
:100AC00020000000420000006F0000006F000000E6
:100AD000740000006C0000006F0000006100000066
:100AE00064000000650000007200000006000000C5
:100AF000FF09000001A10000011900000129000008
:100B00004015000000260000FF00000075080000EE
:100B100095400000810000001901000029400000FC
:100B200091000000C0000000EE8400001885000065
:100B30001C850000508500004572000061730000B4
:100B4000696E0000672000004465000076690000BF
:100B5000636500002E2E00002E000000457200008C
:100B60006173000065200000436F00006D7000009D
:100B70006C65000074650000005700007269000099
:100B800074650000204300006F6D0000706C000071
:100B900065740000650A0000507200006573000073
:100BA00073200000526500007365000074000000AF
:100BB000526500007365000074000000754D000070
:100BC0004F470000493200000A4200004F4F00002A
:100BD000544C00004F41000044450000520000000A
:100BE0000080FB008181FB00000140000281410088
:100BF0004311DD0003A020000301410012F0A10019
:100C00000104E00004003A0000004000A180200040
:100C1000823078000300370000004000E1802000AF
:100C20008230780012E0A1006401410012E0A000CF
:100C300000000600214A800080C0B300E78F50000A
:100C40000E003E0001407800818120009140780034
:100C50000104E00004003A0013C0B30082812000C8
:100C60000349780005003700E1CF500003003A0047
:100C700023C0B30082812000034978004194200002
:100C80000081FB00910811007140800080487800CD
:100C9000A1952000D1408800219420009100780087
:100CA000E1806000030032000004E0000C003A0024
:100CB000000006000004E000110032000294200051
:100CC00092017800D140800093587800D14088008C
:100CD0000309E8000040E900F8FF3A0000000600C0
:100CE0000294200092017800D1408000935878004F
:100CF000D14088000309E8000040E900F8FF3A000D
:100D00000000060000C8B30021952000914F10009C
:100D100033003A0001CCB300209420000148780051
:100D20005095200010407800E24F5000090032003A
:100D3000E34F500019003200E14F500026003A0006
:100D4000C04D2800004A880020012000204A880069
:100D500000000600409520001004E0000C003A005E
:100D60001080FB000000400041592800610078001D
:100D7000004A880041942000204190008248780079
:100D80008100E800304090008048780000000600B4
:100D9000209420000048EB00000006004095200051
:100DA00021C0B30090CF100008003E001080FB006F
:100DB000000040006159280061007800004A880066
:100DC0001080FB00204A88000000060020942000CC
:100DD0000048EB0000000600209420000048EB00D3
:100DE000000006000040EB00A1952000804878003C
:100DF0008100E800804878002095200010407800AD
:100E00007F4060000080FB00E10F50000B003200CB
:100E1000E20F50000C0032000000E00028003A0011
:100E2000209420001070A0000348E200240032004B
:100E30000100E9001014A0002100370020942000D8
:100E40001070A0001E003700209420001070A00039
:100E500060952000104078006F406000180032005C
:100E6000609520001004E000070035001040780075
:100E70006F4060000080FB0000004000A180200067
:100E8000E1007800070037006095200010407800EE
:100E90006F4060000080FB0000004000E180200007
:100EA000E10078000040280091006000808F500031
:100EB00003003A0011C0B300A0952000014878005B
:100EC000000820002194200011006000070032007B
:100ED000A0952000004A8800010078001000A000C2
:100EE00021C0B3000080E80001487800000006003F
:100EF000AA24AB0011003200A040800010419000F5
:100F000001C8B300814F51000B003A0071408000CE
:100F10001141900041C8B300814F510006003A00D2
:100F2000C1C0B30011409800A040800090409000E4
:100F30000174A00011409800AA24A9000008200014
:100F40005024880000000600881F78007040800050
:100F5000100478004E44DE00614464000020A200CA
:100F60007040880030408000E80F50000B003A00CD
:100F7000409520001080FB00F007B200B0248800EC
:100F80009604E20003003200000120003040880097
:100F900002003700400020003040880019C8BF0020
:100FA000E14F500021003A00A195200070408000E0
:100FB000110098001FFF070018C8BF00E24F500043
:100FC00008003A0041C0B300704080001140980012
:100FD00070408000904090000174A0001140980083
:100FE000200037000804E00008003A0081C4B30084
:100FF0007040800011409800704080009040900048
:101000000174A000114098001600370081C0B300A1
:101010007040800011409800704080009040900027
:101020000174A000114098000E0037008094200049
:101030001004E0000A003D00514A8000C808DE00AC
:10104000640040001080FB004800DD00008070005C
:101050000100320000000100809420001070A10007
:101060001968EF004F047800000006000468EF00E4
:101070000001EB008200780040072000ED0507002A
:101080008284A90000012000002488000968EF0084
:10109000000006008284A80000012000502488007F
:1010A00010C0B30004E8B7000968EF000001EB00CE
:1010B0008200780050072000DE053700889FBE00C0
:1010C0004095200011C0B30090CF10000E003A00F0
:1010D0000080E900104078007F4060000A003A007C
:1010E000209420001070A0003095200032C0B30082
:1010F000904F110003003A000140780003E8B70068
:10110000010037000368EF00409520001004E00064
:101110009C003A000080E900104078007F406000A9
:10112000E24F500097003A00609520001040780090
:101130006F406000930032006095200010407800FE
:101140006F4060000080FB00E10F50008D003C000C
:10115000000220000608E3008A003A0020942000E4
:101160001070A000609520001004E0000C00350015
:1011700010417800EF4061008180FB0081804000D9
:10118000A280200062847800104078006F406000E8
:101190000080FB0001952000E14478000C0037003E
:1011A0006095200010417800EF4061008180FB00D5
:1011B00081804000E2802000628478001040780046
:1011C0006F4060000080FB00E1942000E144780063
:1011D0000908A30002003A000820A100010037001E
:1011E0000820A000609520001004E00007003500F2
:1011F000104078006F4060000080FB00000040005D
:10120000A18020008830780007003700609520001A
:10121000104078006F4060000080FB00000040003C
:10122000E1802000883078003095200031C0B30084
:1012300090CF10001A003A001800E00013003D00A3
:10124000630040001004E000080035001040780002
:101250006F4060000080FB00019520006141780034
:101260000214A0008270780008003700609520000A
:10127000104078006F4060000080FB00E194200087
:10128000614178000214A0008270780098409000BC
:1012900040C8B30000C07000104498003900370007
:1012A000880078000120A2001100E00008003D0045
:1012B000114090000074A1000064A00090409800CC
:1012C00022002000500020005A05070003003700CC
:1012D000114090000064A000904098000918A300FD
:1012E00002003A001800E0001B003D00609520005D
:1012F0001004E00008003500104078006F406000E6
:101300000080FB0001952000614178000214A100DB
:101310008270780008003700609520001040780047
:101320006F4060000080FB00E19420006141780084
:101330000214A1008270780018409000B043B200FF
:1013400010449800220020008800780050002000FF
:10135000380507000300370018409000B043B20082
:101360001044980060952000104078006F406000A5
:101370000080FB0000004000A14A20000100400066
:101380001014A1004F04BE0000000600881F780062
:10139000209420001070A000AC24EF0008A02000D2
:1013A000020220008000EB00080078007BFD0700AF
:1013B0009424A8000040EB00E194200080487800CD
:1013C0000195200080487800F19420008048780042
:1013D00011952000804878001268EF009424A9003D
:1013E0006800440070408800A8408800B840880029
:1013F000409520001040780008E8B7000004E000A5
:1014000003003A0000012000304088000600370049
:1014100012002000818020000200780005050700EE
:1014200000022000304088004F04780000000600D1
:101430002095200001C6B30010C060003F003A00B4
:10144000309520001080FB008000EB00EB0F500077
:10145000E08F580039003E00006001001C0037009A
:101460001C003700350037001A0037003300370002
:10147000060037000A0037002C0037000A0037004A
:1014800008003700140037002000370020942000A7
:101490001070A0008000200030408800000006008E
:1014A00018FE3700B9FF370080802000004A88000E
:1014B000209420009000780013C0B3000081E80061
:1014C000034978001108B300010878000000060005
:1014D00044FE3700F9FE3700609520001081FB00C4
:1014E0002181200000942000010841000080E800D4
:1014F0009000780013C0B3000081E8000349780031
:101500001108B300010878000000060020942000B4
:101510001070A000609520009080FB0020812000CA
:101520004295200092707800000006000001EB0058
:101530008200780020002000BE04070000000600A2
:101540009EC0A9000080EB00702488005024880011
:10155000AA24EF00AC24EF002000200030258800F2
:10156000A824EF008644A900F00920008024880008
:101570006024880082C4A8008804A80000A020007D
:10158000C800DE00C12488000008EB00301078009D
:101590006000B8002050880031508800405088001A
:1015A0005150880060508800715088008050880039
:1015B00091508800A0508800B1508800C050880029
:1015C000D1508800E0508800F15088009424A80091
:1015D0009624EF0094A4A9009424A9008000200080
:1015E000502488008A64AB00FCFF3A000040EB0006
:1015F0002194200080487800819420000081FB0025
:10160000820878008180E80002F02F0091086100D4
:1016100013C0B30002822000034978001282200028
:10162000034978000268EF000068EF000468EF00EB
:101630000A28EF00E19420008048780001952000FE
:10164000804878001028EF000C28EF00F19420006B
:1016500080487800119520008048780080A0200004
:1016600070408800D0002000502588002095200080
:101670001050880081C0B30000A02000014878000D
:101680000000E80041C0B300014878001074A000D9
:101690000868EF002228EF002428EF000968EF0017
:1016A0000628EF0000000600889FBE008A1F780011
:1016B00000457800814478000984FB000838A300C5
:1016C000030032008040EB000A40780044FD070030
:1016D0000828A3000300320011C0B3000A407800BC
:1016E0003FFD07000A85FB000A054500A04A2000CF
:1016F00009707D004F0578004F04BE000000060011
:101700000104E000050032000082FB0004024200F8
:10171000E580200065027A00040037000082FB00AB
:1017200004024200A580200065027A008002EB00DE
:101730000400E0001A00320012029800034A780008
:10174000144190000244B2001242980014419000EB
:101750000234A00012429800144190000274A000CC
:10176000124298000104E000070032000080FB00F4
:1017700000004000E1802000008040001020A20016
:1017800084027800060037000080FB000000400063
:10179000A1802000008040001020A2008402780078
:1017A00005007800000006000004E00014003A0084
:1017B00081C0B300B040800001487800B040800094
:1017C0002195200011009800C1C0B300114098007D
:1017D000B0408000904090000174A000114098003B
:1017E00041C0B300704080001140980070408000FC
:1017F000904090000174A000114098000000060085
:101800008180FB000080FB00000040000080400061
:101810004300DD0002A0200082014000134290003E
:1018200041C8B30001427200944198006400400036
:10183000020040001041900081407100114098006A
:101840000000060094A4AB00190032000080FB00E9
:1018500000004000E18020000080400090007800FF
:101860001103BE00040420000500200006036200EE
:101870008003EB008688BE00900078001103BE0054
:1018800084186B0085906B00900078000120A20006
:1018900001087800914190000344B2009340980001
:1018A000100078009040900004C168001240980039
:1018B000000006002048E2002A003A0010C0B300F1
:1018C00020E8B7002148E20026003A0021E8B700EE
:1018D00019C8BF00E24F50000A003A007040800073
:1018E0000048EB0081C4B3007040800011409800B4
:1018F00070408000904090000174A000114098005A
:1019000000000600E14F500016003A001E68EF008C
:1019100080C0B300A140800080487800A2408000D1
:10192000219520001101980043C0B3001341980095
:10193000A2408000924190000374A00013419800DF
:1019400014C0B300E381200084497800B2408000D5
:1019500000497800B04080001100980001C8B30031
:101960001140980000000600A0408000104278005E
:10197000414A8000C808DE00A09420001080FB00CF
:101980004800DD00008070008480FB00808F5000E4
:1019900001003600004278008480FB000100500006
:1019A000819420004801DD00F30F20009181610047
:1019B000828871004800DE008180E800804878005D
:1019C0000404E000090032000000EB0061942000F4
:1019D00011017800A3952000634978008208E8008F
:1019E0000000E800804F5200F8FF3E00414A8000AE
:1019F000C808DE00A09420001080FB004800DD0035
:101A0000008070001900320081C0B300B040800037
:101A100001487800A1952000B04080001100980096
:101A2000A040800010E8A30008003A0081C4B30081
:101A3000B040800011409800B0408000904090007D
:101A40000174A000114098000000060081C0B3009E
:101A5000B040800011409800B0408000904090005D
:101A60000174A000114098000000060081C0B3007E
:101A7000B040800001487800B040800021952000EF
:101A80001100980041C0B30011409800B0408000A0
:101A9000904090000174A00011409800514A8000CD
:101AA000C808DE00C09420001080FB004800DD0064
:101AB00000807000010032000000010080942000CE
:101AC0001070A1000148E20001003A0079FF070010
:101AD0000000060019C8BF00E24F500001003A00A4
:101AE000A1FF37001968EF001E48E2000D003A0020
:101AF00081C0B300B040800001487800B040800051
:101B00002195200011009800C1C0B3001140980039
:101B1000B0408000904090000174A00011409800F7
:101B2000000006001E68EF00000006000268EF00DB
:101B30000068EF0019C8BF00E24F50000D003A00E6
:101B400081C0B300B040800001487800B040800000
:101B5000A19520001100980081C4B30011409800A5
:101B6000B0408000904090000174A00011409800A7
:101B700000000600809520001080FB009195200059
:101B80009180FB00C808DD008100700040942000B7
:101B9000908F500007003100809520009080FB005E
:101BA0000000E8001081FB004811DD004094200097
:101BB000010871001FFC0700A19520007040800003
:101BC0001100980081C4B30070408000114098005B
:101BD00070408000904090000174A0001140980077
:101BE0000000060094A4A900000820002194200011
:101BF000110060001F003A00809420001004E000F3
:101C000008003D0020C0B30019E8B7000048E2001A
:101C100001003A00C5FF07002168EF002068EF00CF
:101C20000000060081C0B300B04080000148780089
:101C3000B04080002195200011009800C1C0B30081
:101C400011409800B0408000904090000174A000C6
:101C50001140980041C0B3007040800011409800CE
:101C600070408000904090000174A00011409800E6
:101C700000000600209520001004E0000A003D004E
:101C800010C0B30019E8B7000248E20001003A00B2
:101C9000A6FF07002168EF002068EF000148E2007E
:101CA00014003A0003FF370020C0B30019E8B70062
:101CB00081C0B300B040800001487800B04080008F
:101CC000219520001100980041C0B30011409800F8
:101CD000B0408000904090000174A0001140980036
:101CE0002168EF002068EF000148E20001003A009F
:101CF000F0FE0700000006001868EF000168EF0022
:101D00000268EF000068EF001E68EF001968EF003E
:101D100070408000904090000174A1001140980034
:101D2000704080000020A200704088009040900029
:101D30000174A100114098000E48AA00B040800034
:101D4000904090000174A100114098002094200060
:101D50000048EB008000EB00214A880080942000BE
:101D60008180FB00010878000080E80001F02F006E
:101D700010886000AEFD07000001EB0082007800D3
:101D800030002000AB02070096FF3700D0C2B3003E
:101D90001FE8B700C1812000914078000100780061
:101DA000B00FB20013003A00C10FB20000A0200033
:101DB00080804000A1408800010078000020A2003F
:101DC000B040880002C023001101610000402300E0
:101DD000800F510006003A0011009000219520006C
:101DE00007000900B05878008000B100C2FF37003A
:101DF00038FF3700E80F500001003A0052FC07009E
:101E00000000060010418000214180006100400078
:101E1000E080480010418800214188000448E20029
:101E200004003A000948EC0009E8B70001003A0054
:101E300009E8EF0000000600881F780030408000AD
:101E40000000E00012003A009424EF008C24EF0020
:101E50002000200030258800A824EF008644A90037
:101E6000F0092000802488006024880082C4A80033
:101E70009404AB0003003A009404A8009404AB005F
:101E8000FDFF3200100020003040880002003700C3
:101E9000E10F500008003A0094C4AB0006003A007D
:101EA0008AA4EF008C24EF008C04A8008C84A80086
:101EB00020002000304088008084AB000500320004
:101EC0008284AB000300320000012000002488005F
:101ED00066FC07008824AB00020032008EC0A90017
:101EE000690037008A04AB00070032008C04AB00A5
:101EF0000500320092FD07004000200030408800BD
:101F000010002000502488008A84AB0003003200B7
:101F10008C84AB00010032005EFC070080C4AB0083
:101F2000030032000004200000248800B5FF0700F1
:101F30008A44AB000E0032008C44AB000400320037
:101F4000120020008000EB0030072000390207005B
:101F500040002000502488001FC8BF00030032004A
:101F60000040E9001FE8B70001003A0051FE0700F9
:101F70008AE4AB00030032008CE4AB0001003200C5
:101F8000DBFB07008A24AB00090032008C24AB0085
:101F900007003200120020008000EB00F0FF270055
:101FA000240207008EA4EF002000200050248800A7
:101FB00030408000E30F500002003E008EC0A900B8
:101FC000310037008C64AB002E00320048C0B300F3
:101FD0008A64AB0003003A002A0037008A64AB0031
:101FE0002800320091248000C08120000148780040
:101FF0000181FB004411DE000240780002427800BB
:10200000D381200084497800820020005224880077
:102010000138A30009003A008080FB0002952000EF
:10202000E2C1780061C261000404A2000304A100BF
:1020300084C1710003F17800080037008080FB0044
:10204000E2942000E2C1780061C261000404A200B1
:102050000304A10084C1710003F178000004E000D2
:1020600002003A0049FF0700040037000001EB00BE
:10207000C181200020072000EE0107000844E9008C
:10208000D6FF3A008EC0A9004F0478000000060079
:10209000104180002141800000000600881F780068
:1020A0002628EF002828EF0090CAB3002AE8B700DE
:1020B00000802A00604188002000200070418800D4
:1020C00018C0B30008407800818320008848780059
:1020D0003068EF0034A8EF0036A8EF003268EF0058
:1020E000D1C1B30070FD070003C4B300028C20000F
:1020F0008040EB000840780081FD070030418800F7
:102100004F0478000000060012832000124178007E
:102110000281FB008001EB004A18DD00C610DE00E2
:10212000810070004A10DD0022042400023B880078
:102130008141780022032000034978000081EB00F0
:102140000208BB001000FC0050052000303B880056
:10215000A00A2000303B880061E7A80000000000D2
:10216000000000006007E200FEFF350000000600EE
:1021700030002400003B880032C8BF001D00320040
:10218000019020000081FB008001EB00A441800051
:10219000B54180000201520083815A000342780059
:1021A0002003200004487800020078001108BB00DA
:1021B000110190000288BB001000FC0050052000B7
:1021C000303B8800A00A2000303B880061E7A8006F
:1021D00000000000000000006007E200FEFF350084
:1021E00032C8ED0032E8B700E48040000004E000AF
:1021F000E4FF3A0061C7A9000000060023032000A5
:1022000093417800400ADE00050020000443780076
:102210002203200006497800000178001282BA00EB
:10222000840078001200BA000342780022032000E4
:102230000449780000000600889FBE008A9FBE0007
:102240003048E20022003A00404180000000E000F7
:10225000020032001000E0007301350030418000C0
:102260000000E00005003A00F08B2000F183200020
:102270000204200000014100030037001000E000CC
:10228000F9FF3D0068013700D0687800820F5000E8
:10229000FDFF3A0003C4B300028C20008040EB0035
:1022A00010C0B30016FD07003041880010C0B30015
:1022B00030E8B700F0872000010420008080400053
:1022C0000068EB00810F5000FDFF3A005601370017
:1022D0000084200010407800E54F5000910032004B
:1022E00006003E00E34F50005A0032006E003E00F0
:1022F000E24F50004C013A0006003700E74F500013
:10230000E6003200DB003900E84F500046013A0099
:102310003A01370020C0B3000188200080487800CF
:1023200082C3B3008100E800824878008100E800A1
:102330008048780011C0B300308820000148780040
:102340000040EB00418820008048780082C1B30043
:102350008100E800824878008100E8008048780029
:102360008100E8008048780000802E00F1FF2F00F7
:102370006241800073418000020040008380480079
:10238000F20F200083882000824960004802DE00AE
:102390008301E800844978008301E80082C9600075
:1023A000C808DE000300E800014878000000E800EB
:1023B00000C8EB003848E20019003A0031C0B30011
:1023C000014878000040EB0082CFB300E380410079
:1023D00082487800B2CAB3008100E80082487800E1
:1023E00022C0B3008100E800824878008100E80044
:1023F0008048780082C0B3008100E80082487800FD
:102400008100E800804878008100E800804878007A
:102410008100E800804878000100E80000C8EB0077
:10242000404180000000E000020032001000E000A7
:10243000FD00350003C4B3000288200011C0B300C2
:1024400001407800AEFC0700404188003068EF0092
:10245000F5003700108420001004E00008003A0066
:10246000A0CAB3002AE8B70083BF2A0063418800EE
:1024700023002000734188003868EF00080037000F
:1024800090CAB3002AE8B70000802A0060418800A3
:10249000200020007041880010C0B30038E8B70069
:1024A0003068EF00E00037008000EB0010002000F3
:1024B00010010700C05928005601070060C0B30092
:1024C00031E8B7002AC8BF000080FB000000E80028
:1024D000E60F50000B0034000BFF070056FE07000C
:1024E0003148EC0031E8B7000080FB00A1822000F9
:1024F000914078008180FB008100E800810F50004E
:10250000F5FF350061C7A9003068EF008000EB00DF
:1025100010002000F7000700E05A28003D010700E6
:10252000C1003700A0418000B1418000E10F4000B0
:10253000E08F48000E003A00128420001281FB0058
:10254000238420009381FB00C819DD000300710083
:10255000328420001281FB00438420009381FB0021
:10256000C819DD0083007100A0418800B1418800D6
:10257000128420001281FB00238420009381FB0041
:10258000C819DD0003007100328420001281FB00B5
:10259000438420009381FB00C819DD008300710093
:1025A000A2418000B3418000820F5000838F580009
:1025B0002E003A005084200010407800E14F500077
:1025C0002A0036000044EB0021832000914078006F
:1025D0000181FB00820141000080FB00820320009A
:1025E000000051004F01DE00000041000081D100D9
:1025F0000880FB0000004100640040000000400033
:1026000002842000624278000482FB000000410046
:10261000104190004811DD0002017200009020007E
:1026200002B079000140E80032E8B700A241800022
:10263000B341800061014100E0814900A24188006E
:10264000B3418800FC4F500001003A00C8FE07006B
:102650000844E80050842000104078008080FB008F
:102660008100D100814F5400D7FF39003068EF005E
:102670006D003700BEFE070034A8EF0036A8EF005B
:102680003068EF008000EB00100020009900070088
:10269000D05B2800DF000700630037004041800066
:1026A0000000E000020032001000E0005E00350093
:1026B00071C0B30000882000014878001284200017
:1026C0001281FB00238420009381FB00C819DD00E8
:1026D00003007100328420001281FB00438420003B
:1026E0009381FB00C819DD0083007100F20F200008
:1026F00013882000824960004802DE008301E80060
:10270000844978008301E80082C96000C808DE00BF
:102710000300E80001487800508420001040780051
:102720008380E80080487800E14F50002B0036009D
:102730000044EB000881FB008001EB0014842000C2
:102740001482FB00258420009582FB00C82ADD004E
:1027500005007200348420001482FB0045842000B0
:102760009582FB00C82ADD0085007200020040004F
:1027700083804800A1FE07008884FB005484200069
:102780009482FB008502D1008583FB0007855400FD
:102790000A02B000068820000A0545000A05430029
:1027A000F40F2000044D6000C805DE001B459800B2
:1027B00081016200078054001002B0000000400058
:1027C0000000430004C86100C818DE0011409800F2
:1027D00008C4E80088CF5200D6FF3E0003C4B3000F
:1027E0000288200011C0B30001407800C4FB07003C
:1027F000404188003068EF000B0037008000EB009C
:10280000100020003B000700805D280081000700C9
:102810009424EF000080EB00000000000000E900BD
:10282000FDFF3A000000FE004F05BE004F04BE0051
:102830000000060031072000810F50000D0032001B
:1028400005003C00E10F500010003200E30F500083
:1028500011003A000F00370041072000810F50009F
:10286000080032008100E800810F50000A003A00A1
:1028700002003700FE00070007003700FC000700D9
:1028800005003700FA0007000300370003FE0700C9
:10289000010037007100070010000500EC22A800BD
:1028A000000000000000000000000000EC22A90071
:1028B0000000060000F02F00E022B600F002A900A0
:1028C000F022A900E822A900F402A900F422A9003C
:1028D000EC22A900000006000000FB0001F02F0020
:1028E000221780008280600080807000211788009D
:1028F0000000060080417800F00F2000E022B700C1
:10290000F422A800F402A900EC22A80000000000B4
:10291000000000000000000012178000EC22A90057
:102920000278A300F8FF3A0002F02F00002E2000EA
:1029300010086100F422A9008180FB008100EA00F8
:10294000CF08DE00A21780000200A1000281700003
:10295000A217880003407800DFFF0700CFFF370091
:10296000D4FF070000202100A10720001801070064
:102970008040EB0080C3B300DEFF07008040EB0027
:1029800080C0B300DBFF07008040EB0010C0B30045
:10299000D8FF07008040EB0060C0B300D5FF070000
:1029A0008040EB00C0C0B300D2FF070000B82B008E
:1029B0000100200006013700F0F32F004427B60085
:1029C00042A7AB0003003A000000000042A7AB00A2
:1029D000FDFF320040A7A900F0C2A900D022A80044
:1029E000DFFF07000000EB00E3000700D4FA070058
:1029F0000060FE0010FD070030408000FF0F500017
:102A0000FBFF36008824AB00F9FF3A000AFE0700FE
:102A1000F7FF3700881F780000047800184078001E
:102A20000004E0000B003200EA4F500004003A00BE
:102A30008040EB0000CCB300AEFF0700020037007F
:102A400011C0B300ABFF0700584078000004E0005D
:102A5000F5FF3A004F0478000000060020952000A2
:102A6000104078007F406000E14F500054003A0071
:102A7000609520001004E00051003A00630050000F
:102A800061C0B30090CF10001B003A000080E80046
:102A900010407800FBC04000814F5000040032001D
:102AA0008140E800814F500013003A000B003700CE
:102AB00008C8BF00E14F50000F003A000050280046
:102AC000004A880090002000204A880001CCB30012
:102AD0002094200001487800070037006057280044
:102AE000004A8800D0012000204A880001CCB300B1
:102AF00020942000014878002095200002C6B300F1
:102B00009040610000C2B30080CF50002C003A001A
:102B10003095200010407800E34F5000190032003B
:102B200003003E00E24F500025003A000500370048
:102B3000EA4F50000B003200EB4F500020003A00EB
:102B400018003700A0832000004A880010002000F1
:102B5000204A880011CCB30020942000014878005E
:102B60000000060001C8B30020942000014878004E
:102B70005095200010417800A18320008248780001
:102B800000000600B0832000004A880010002000EA
:102B9000204A880011C8B300209420000148780022
:102BA0000000060001C8B30020942000014878000E
:102BB0004095200010417800B183200082487800C1
:102BC00000000600E10F500003003200E20F500049
:102BD00004003A0002003700F4C2A800000006001A
:102BE000F4E2A80000000600E10F500003003200EC
:102BF000E20F500004003A0002003700F4C2A900BE
:102C000000000600F4E2A90000000600E10F5000F9
:102C100003003200E20F50000B003A0005003700BD
:102C200000042000F402B6000000EA004F00DE00BD
:102C30000000060000082000F402B6000000EA00D0
:102C40004F00DE000000060000000500E10F50000C
:102C500003003200E20F500004003A000200370087
:102C6000F0C2A90000000600F0E2A9000000060082
:102C70008824AB000200320010002000DAFF370089
:102C8000000220000608E30010003A00F041800036
:102C9000E10F500002003A00CAFF07001A00370097
:102CA000B1042000810F500003003A001000200002
:102CB000CDFF07001400370061092000810F50008C
:102CC000110036003E28EF000F003700F041800071
:102CD000E10F500002003A00BAFF07000A00370077
:102CE00021032000810F500003003A001000200053
:102CF000BDFF070004003700613B2000810F50003A
:102D0000010036003E28EF003E28EC0000000600DF
:102D10004009000022000000000000000008000040
:102D20002600000000000000000A00002000000053
:102D3000000000003A08000002000000000000004F
:102D4000400800000001000000000000260800000C
:102D500014000000000000003C0800000200000019
:102D600002000000010000003E0800000200000018
:102D700000000000000000000000E00013003A0026
:102D800083E0A800100020002700070010002000AA
:102D90001D0007000004E00006003A003008200093
:102DA0004007B6000300320083E0A900001A0400C7
:102DB00000000000E05D280016FF07001000200062
:102DC000A2FF070020002000A0FF0700000006006F
:102DD000F03FB1000180B10006003500EE030900AC
:102DE00000000000403FB1000180B100FBFF3D004A
:102DF0001000B000203FB000020035000080090044
:102E00000000000000000600E10F500005003A003D
:102E100090168000620060000000E9004F00DE00B4
:102E20000000060000000500E10F500001003A001C
:102E3000D022A80000000600FFFFFF00FFFFFF00F8
:10340000101B040000000000241D04000000000048
:10341000241D040000000000241D04000000000022
:10342000241D040000000000241D04000000000012
:10343000241D040000000000241D04000000000002
:10344000241D040000000000D81B04000000000040
:10345000241D040000000000241D040000000000E2
:10346000241D040000000000241D040000000000D2
:10347000241D040000000000241D040000000000C2
:10348000241D040000000000241D040000000000B2
:10349000241D040000000000241D040000000000A2
:1034A000241D040000000000241D04000000000092
:1034B000241D040000000000241D04000000000082
:1034C000241D040000000000241D04000000000072
:1034D000241D040000000000241D04000000000062
:1034E000241D040000000000241D04000000000052
:1034F000241D040000000000241D04000000000042
:10350000241D040000000000241D04000000000031
:10351000241D040000000000241D04000000000021
:10352000241D040000000000241D04000000000011
:10353000241D040000000000241D04000000000001
:10354000241D040000000000241D040000000000F1
:10355000241D040000000000241D040000000000E1
:10356000241D040000000000241D040000000000D1
:10357000241D040000000000241D040000000000C1
:10358000241D040000000000241D040000000000B1
:10359000241D040000000000241D040000000000A1
:1035A000241D040000000000241D04000000000091
:1035B000241D040000000000241D04000000000081
:1035C000241D040000000000241D04000000000071
:1035D000241D040000000000001D04000000000085
:1035E000241D040000000000241D04000000000051
:1035F000241D040000000000241D04000000000041
:10360000241D040000000000241D04000000000030
:10361000241D040000000000241D04000000000020
:103620000FC320000E7F24000E0188000000000060
:10363000000020000000E000020032000001200035
:103640002002880014000700430107000000E0008A
:1036500003003A00E00C25000100200002003700C2
:103660000000200001002000810F700001003200E6
:1036700014000700000020000000E00002003200FB
:103680000000020000000000C6410200000000002F
:103690000040DA000000FE004440A900601A20004B
:1036A0000000E0000300320000002000A0018800BC
:1036B0004440A800000006008A1F78008B1F780095
:1036C0000000060091018800800478000000EB00F3
:1036D0001A003700E284440032A0B4009905BA0011
:1036E000E284440032A0B4009906BA00E2844400A7
:1036F00032A0B4000006EB00476FDE00FD07B20009
:10370000636CE10003003A00EBFF07000000EB00F0
:103710000A003700606CE10004003A00005DEB0035
:103720008B05E900FDFF3E00040037006168E10001
:10373000010032000086EB000B00070019C7BA0039
:103740001905BA000E04E00003003A000A00E00088
:10375000E0FF3A0000000600FE07B2009E0188006C
:103760008A047800F5FF3700395DBA008B05E9005F
:103770000C003200295DBA008B05E9000800320018
:103780000C00E00003003A00E284440032A0B400E0
:10379000F5FF370019DDBA008B05E900FAFF3A00A2
:1037A0008904E800E184440032A0B400000006006F
:1037B0003600F800809FBE00829FBE00849FBE003E
:1037C000869FBE00881F78003400F80000002000AB
:1037D000A00188000800FA008040EB0010C0B30090
:1037E000891907000E0078001E1C070081A7200021
:1037F00006000900BE5878007E00B10098418000A4
:1038000087418000408320005001BE004000BE0080
:10381000E4A72000144278000483FB00D4A7200012
:10382000144278008482FB00C4A720001442780070
:103830000482FB00881F7800871F7800809FBE00ED
:10384000829FBE00861F7800851F7800841F780045
:10385000F0FF2A00801F780080A220006602070087
:10386000F487570080A220009E1907004000200026
:103870008612070080418800500020008312070054
:1038800090418800AE17070044832000009ABE00D4
:103890000292BE0080418000B00C8800901680002B
:1038A000620060000000E0002F003A0090168000E7
:1038B000680060000000E0002B003A001117800053
:1038C00000102000008060000000E00026003A00A8
:1038D0001117800000202000008060000000E00040
:1038E00021003A0000A8200031C0B3000148780050
:1038F000804180008040780010A8200001487800B6
:10390000804180004880DE008040780020A82000B0
:1039100001487800904180008040780030A8200065
:1039200001487800904180004880DE0080407800A7
:1039300040A820000148780050A82000C1CFB30063
:10394000014878001FC8BF000004E00003003A00EF
:1039500061C0B30000A82000A815070030022B00AA
:10396000601907001C003700E0418000E10F5000A3
:1039700019003A001FC8BF000004E00016003A001A
:1039800080418000CF80DE00130107006022B80074
:103990000600200007092400700007006466260066
:1039A0006566260066662600A70024000E01070053
:1039B000849E2000809FBE00829FBE0070022B006C
:1039C000801F7800040078000B020700EA87570088
:1039D000809E20009C1507008460A9000080FA00EA
:1039E0003400F9004F0478004F03BE004F02BE00C0
:1039F0004F01BE004F00BE003600F9000040060037
:103A00003600F800809FBE00829FBE00849FBE00EB
:103A1000869FBE003400F80000002000A00188004E
:103A20000000FA00AA0A07000080FA003400F9003A
:103A30004F03BE004F02BE004F01BE004F00BE004C
:103A40003600F900004006000040DA000000FE00E9
:103A50000A00FA00E20F500034003E00F05E8000E1
:103A6000E10F500003003200E20F500011003A0055
:103A70000C003700032220000300E00001003A00A0
:103A80000040DA002002E200020035002822EF00A8
:103A900021E2A8002342AB000D003A002342A80017
:103AA0000B003700032320000300E00001003A0070
:103AB0000040DA003002E200020035003822EF0058
:103AC00031E2A8003342AB0001003A003342A800C3
:103AD000820178000B0037003102FB00E10F50003B
:103AE00004003A002322AB00FEFF3A0024118800B4
:103AF000030037003322AB00FEFF3A00A411880018
:103B00008301E9000300E000F3FF3A00E10F5000F9
:103B100003003A002302AB00FEFF32000B00370027
:103B20003302AB00FEFF32000800370033002000F4
:103B3000B3BF9F00C0BF9F00D1BF9F00E2BF9F00E7
:103B40006A805700F00707006FB9970002007800FD
:103B50000080FA0000000600000005002800FA00BE
:103B6000889FBE008A9FBE008C9FBE0003866B00AC
:103B7000800007006400E100440032006408E100B6
:103B80004A0032006100E100460032006108E100B5
:103B900049003200EC0647006000B8003D02BE005C
:103BA0003D03BE00F48657006011B8003D04BE001E
:103BB0003D05BE007D0320000B0037000000A00083
:103BC0008D06E900130032000402420085824A009B
:103BD00006034B0087834B000000400081804800B3
:103BE00002014900838149000802520089825A007B
:103BF0000A035B008B835B00F0FF3B00080242007E
:103C000089824A000A034B008B834B008D06E90032
:103C1000EDFF3A008482720086827200F707B200DC
:103C20008782720001003200150020001E049000FF
:103C30003E0B900006035400E63FB0000368A3006B
:103C4000070032000000A7000500A0008301D1009A
:103C50000281D3008180D3000080D3000603E800F6
:103C60008301D1000281D3008180D3000080D30082
:103C70000002EB000482D2001200070003F0A10052
:103C80000CF0A70003F0A0004E00370064024700CC
:103C90006408E100480032003400BE003401BE0078
:103CA000F6FF37006108E100430032006011B80000
:103CB0006000B800F1FF370003FF2700020020007A
:103CC000FBFF3700180020005700200008045300B5
:103CD0000D003D000600200097FC2F000740E1008A
:103CE0001E00340084827200610260008301D100F2
:103CF0000281D3008180D3000080D3000804E80053
:103D0000F8FF3A00470020006104600005047400D9
:103D1000040464000D00320061004000E0804800AF
:103D200060014900E081490003B8A50007003200A6
:103D30000603E8006538E10004003A008301D10081
:103D40000281D3008180D3000080D300F87F20005F
:103D50000830E10003003500080378006000B80077
:103D60006011B8004433DD00F300B200830173003A
:103D700000000600680447000294BE000094BE00E4
:103D8000FC0447008694BE008494BE0009007800BD
:103D9000A900070008007800A70007009900780034
:103DA000814F70000B003B000800BE00940007002C
:103DB0004F00B10003003700F3FF2700F2FF2F0090
:103DC0006110B9004F06BE004F05BE004F04BE0093
:103DD0000080FA00000006004F89DE0082017800B2
:103DE000BC003700000000002800FA00889FBE00D9
:103DF0008A9FBE008C9FBE0003866B00DDFF07001C
:103E00000028A30064003A000128A30067003A00DC
:103E10000008A30062003A000108A30065003A0010
:103E20001E009000BE08900081064000ED3FB100EA
:103E3000F4805700EE019000111AB8008E0990002E
:103E4000311BB8009E099000311CB800511DB8000C
:103E5000F485570046000700FE0190003A00070075
:103E60008B85E8003E0007008E09900040000700A7
:103E7000EE019000340007008B85E8003800070051
:103E80008E099000400007009E0990001B18B800A2
:103E9000890440000A854800FE01900034000700B4
:103EA0008B85E80038000700EE0190003000070025
:103EB0008E0990001B18B800890440000A8548004C
:103EC0000A98A30008003A000402420085824A00D2
:103ED00006034B0087834B0008044C0089844C0088
:103EE0000A054D008D06E900848272008502730088
:103EF0004C3ADD00850272000100320015002000FE
:103F0000443ADE001400B2004538DE00CB45DD0047
:103F10000B007000C540DE00CB4DDD008B807000D3
:103F20004549DE00CB55DD000B017100C551DE00B7
:103F30000D03780063FF070003F0A1000CF0A70059
:103F400003F0A0009FFF37001B18B8008502400057
:103F500006834800E0834B0060044C0007003700F4
:103F60001B18B8000603400087834800FAFF37009B
:103F70001B18B8008703400008844800E0844C0008
:103F800060054D00000006001B18B8000804400042
:103F900089844800FAFF37000108A30086FF3A0031
:103FA0005800BE005801BE00E3FF37000008A30020
:103FB00081FF3A0009047800F9FF37000000000093
:103FC0006022B800060220000000D0008180D200EC
:103FD0000482D2008582D2000000A00002025200BA
:103FE00083825A00030031000202420083824A00A9
:103FF0000000A1000603E900F3FF3A0000000600FC
:10400000E48240001078A300070032006402400000
:104010001178A3003400BE001401BE000400320079
:104020000330A700000006003500BE001501BE00E9
:104030000330A00000000600800078005002BE009F
:104040005003BE004439DE00F700B200F37F2000C9
:1040500003016100090032000218E10016003A0075
:1040600085017200830173008381730000082000C2
:1040700015003A004000200013003700850172004F
:10408000830173008381730005003A0004A8BE0019
:1040900006A8BE00100020000B0037000201E90056
:1040A0000402420085824A0006034B0087834B00CE
:1040B0000748A300F9FF32000740A00004A8BE0093
:1040C00006A8BE0020002000800098009200980002
:1040D00000000600881F7800030478000300E00059
:1040E00007003D0060001000E0801800600119002A
:1040F000E081190002003B0001F02D0003003700B1
:104100000400070008F0A70003F0A0004F047800A7
:1041100000000600889FBE0000827000040271004B
:10412000048271002400320036432000C5002000C4
:104130008383CF000A0039000541B1008283CF009C
:10414000070039000541B1008183CF000400390028
:104150000541B1008083CF00010039000541B10065
:1041600085C353006022B800120032000A003B00F1
:1041700084827200610260008301D1000281D30059
:104180008180D3000080D3000603E8008743E80065
:10419000F7FF3A0007003700000040008180480028
:1041A00002014900838149000603E9008743E900D1
:1041B000F9FF3A00C3FE07004F04BE0000000600EE
:1041C0008001780002003700B15978000201E9004F
:1041D0000200E000FCFF3A000000060080017800C9
:1041E00002003700815978000201E9000200E00076
:1041F000FCFF3A00000006000C00FA00889FBE0099
:1042000000047800F0FF2700D0BF9F008004EB007F
:1042100099BF9F0088BF9F00A8BF9F00200C20006F
:10422000B0BF9F0078815700CFB0970070805700D3
:10423000D00007000FB89700094878008FB89700A2
:10424000088050004F04BE000080FA000000060005
:104250000800FA00889FBE008A9FBE000084FB0011
:10426000D1C6B300814F5000340036004B06200009
:10427000110009000B84D80081057800720040000D
:104280004300DD00898F2000008044006022B800D8
:104290000600200007FE23005001BE004000BE00C3
:1042A000D1FE07000002BE000203BE0084BF9F00D3
:1042B00095BF9F00A6BF9F00B7BF9F00AA00200028
:1042C000110009008A85D80080057800E98545003D
:1042D000C35DDD008B8544003B02BE002B03BE00A6
:1042E0000FB897009FB897002FB99700BFB99700F4
:1042F000BDFE07000002BE000203BE0084BF9F0097
:1043000095BF9F00A6BF9F00B7BF9F001100090087
:104310000A84D800010478004344DD008884440006
:104320003902BE002903BE000FB897009FB897005E
:104330002FB99700BFB997001D003700EA4F500012
:1043400013003600AA002000110009000A84D800DA
:1043500001057800690440004344DD00898F200096
:10436000088444006022B8000600200007FE2300F5
:104370003800BE002801BE009BFE07004355DD004B
:104380008A8444003902BE002903BE0008003700B9
:104390004344DD00808F2000080440006022B80004
:1043A0000600200007FE23003800BE002801BE00E2
:1043B0008DFE07004F05BE004F04BE000080FA00CE
:1043C000000006000800FA00889FBE008A1F7800DF
:1043D00000047800D00620000800E0001F003D0027
:1043E0000804EA00800F5400070034004206200051
:1043F000110009000204D800720040004300DD00F3
:10440000898F20001D003700EA0F5400100034008F
:10441000A2002000110009000204D8000104780065
:10442000690040004300DD00818F200000804000D3
:104430004344DD00888040003102BE002103BE00FD
:104440005001BE004000BE0067FE07003C00370080
:104450004344DD00808F200036003700800F540079
:104460002500340042062000110009000204D80093
:10447000720040004300DD008984200080814400F8
:10448000AA002000110009008A00D8008000FD0069
:10449000E9804000C308DD00818044003102BE0095
:1044A0002103BE003300BE001301BE004EFE070014
:1044B0000002BE000203BE0094BF9F00A5BF9F0084
:1044C000B6BF9F00C7BF9F00110009000A04D800B3
:1044D000010478004344DD00888444003902BE00B2
:1044E0002903BE001FB89700AFB897003FB99700E7
:1044F000CFB99700D4FF3700EA0F54000B00340007
:10450000A2002000110009000204D8000101780077
:10451000690040004300DD008184200000804000ED
:104520004311DD0082804000C3FF37004344DD00BB
:1045300080842000080440003800BE002801BE002E
:104540004F0578004F04BE000080FA00000006000E
:10455000D0019000028151004240A90003003400C4
:1045600010017800014978000208E8000100780095
:10457000000006006F02B000889FBE008A9FBE0048
:104580008C9FBE008E1F780000067800B1AF9F00A0
:1045900092B79F006000B8006011B800D0AF9F00D4
:1045A000E1AF9F00F2AF9F0083B79F008006EB0052
:1045B000C7043700BFA897008100E800B1AF9F0093
:1045C00051C2B300814F500003003A00BFA89700CA
:1045D0000007EB0011003700BC0090000000FB005A
:1045E0000168A300070032000D0178008000780008
:1045F0000C007800D6FF07000000E00005003A003C
:10460000B30437008C007800BD040700E10F4000C0
:10461000AF0432008D06E800AD04370001017800D8
:1046200031407800D3C2B300834F50000C003200F9
:1046300007003C00EDC15100834F50000A003200DA
:10464000EBC14100834F50000D003A0008003700D5
:1046500003C3B300834F500009003A00060037003F
:104660000E30A000EDFF37000E00A000EBFF37007A
:104670000E10A000E9FF37000E20A000E7FF370072
:104680000E18A300010032000E00A1000E38A30096
:10469000010032000E20A1008000FB000103B100E8
:1046A000E98F50000C003E00020078008005EB000E
:1046B0006A59B900B005FB000B03B10082854500C3
:1046C000000178009000FB000103B100E98F500069
:1046D000F7FF3600080037008005EB00A1C2B300E9
:1046E000814F500004003A009FB19700C305780045
:1046F00093B79F000201E800E0C2B300924F1000A0
:1047000016003A000EE0A00064405000D24F1000A6
:1047100003003200020078008001EB00080037003F
:104720009FB297004503780095B79F00E6B79F00BA
:104730000201E8000C0037006A19B90082814000CC
:1047400000017800B000FB000103B100E98F5000C8
:10475000F9FF3600E3B79F00030037000EC0A0004A
:104760008003EB00E7B79F008201780033407800B8
:1047700003017800C1C6B300814F50002B00320006
:10478000B3AF9F0014003C00E8C05000814F5000C0
:104790002400320009003C00ECC05000814F500062
:1047A0002A003200EBC04000814F50008C003200E4
:1047B0000004E0004B043200A200370061C6B300E1
:1047C000814F50001B003200E3C04000814F500079
:1047D0009C003A001300370031C7B300814F5000EE
:1047E0001E00320007003C00E4C05000814F500022
:1047F000130032008140E800814F500091003A00E0
:104800001200370051C7B300814F500092003200B0
:10481000E3C04000814F50008A003A00E0CF9F0083
:104820000C003700E0CF9F008D0037000E40A00045
:10483000CDFF3700E0CF9F000EA0A000880037001A
:10484000E0CF9F000E60A00085003700E0CF9F0002
:104850000E50A0000E70A00081003700E0CF9F0036
:104860009FB097004100780091B79F000004780046
:104870000000E00001003A0028B420008800780021
:104880000000EB00010037000000E8006141780003
:104890000204E000FCFF3A00800478006FB197004A
:1048A0000200E00003003200890F510001003100D6
:1048B000820478000005EB00898F55000100360066
:1048C00009855500680767002A003A001100370083
:1048D0003C0090000068A300070032000D01780042
:1048E000010220000C00780019FF07000000E00022
:1048F00006003A00060037008C0078000002200015
:10490000FF030700E10F4000010032008D06E800C0
:104910000A05E9000A00E000EDFF3A000085EB001F
:10492000140037003C0090000068A300090032002A
:1049300008007800B000FB00000478000D0178004A
:104940000C00780002FF07000000E00008003A00B9
:1049500008003700880078003100FB00010478006F
:104960008C007800E6030700E10F400001003200F0
:104970008D06E800090078008004E9000000E000EE
:10498000E8FF3A000E00E000D103320011003700CA
:104990003C0090000068A300070032000D01780081
:1049A000010220000C007800E9FE07000000E00092
:1049B00006003A00060037008C0078000002200054
:1049C000CF030700E10F4000010032008D06E80030
:1049D0000A05E9000A00E000EDFF3A00BC033700D9
:1049E0009FB197004302780093B79F00CFA2DE00EB
:1049F000482BDD004820DE0000007300C828DE00E0
:104A0000E0CF9F000E48A300080032000004E00041
:104A100006003200E14F400004003200F0CF9F005A
:104A200084D79F002900200002003700F4CF9F00A8
:104A300019002000E7FC2F008F8343000704E800E3
:104A400096FF3700E0CF9F00E8FC2F000F044400E2
:104A50001900200091FF3700E0CF9F000E0CB3003B
:104A60000170200081006700700067000100E00015
:104A70001C0232000EC8A3000200320061002000B8
:104A8000E1B79F001FB19700E80051000000E0006F
:104A90000900320091B79F00810278005503BE00E3
:104AA0004502BE00A4B79F00B5B79F00C6B79F00E0
:104AB000D7B79F000700370091B79F005101BE0094
:104AC0004100BE00A0B79F00B1B79F00C2B79F00D2
:104AD000D3B79F006022B8006033B8002FB09700B2
:104AE000BFB097004FB19700DFB197008604070071
:104AF0000000E0000A003D002FB29700BFB297000F
:104B00004FB39700DFB3970007F0A200A4B79F0050
:104B1000B5B79F00C6B79F00D7B79F003E00B30050
:104B20000000EB0090AF9F006022B8006033B80037
:104B30002FB09700BFB097004FB19700DFB197003B
:104B40007B0407000000E0003400320024FD2F0049
:104B50000F0242002FB09700BFB097004FB19700EF
:104B6000DFB19700AA0407001FA897000000E90022
:104B70006302B900A2002000110009000202D8005F
:104B800090AF9F000000E00002003D000000E9003F
:104B900090AF9F001FAC97000800EA0009FE0700D5
:104BA0002FB29700BFB297004FB39700DFB39700C3
:104BB0008DFC07000002BE000203BE00D4AF9F00C0
:104BC000E5AF9F00F6AF9F0087B79F006022B80057
:104BD0000600200007FF23004B0407000000E00050
:104BE00002003D000804E9000B0037006022B80015
:104BF00006002000470224005FA89700EFA8970056
:104C00007FA997008FB19700440407000000E000DF
:104C1000020035000804E80098AF9F00EFB297004B
:104C2000EC8F52000F003C000540780088FD070023
:104C30000002BE000203BE002FB09700BFB0970075
:104C40004FB19700DFB19700B10307000002BE002B
:104C50000203BE00A4B79F00B5B79F00C6B79F0070
:104C6000D7B79F001FAC9700E90F540015003C0018
:104C70006022B8006033B8002FB09700BFB0970033
:104C80004FB19700DFB19700290407000000E00052
:104C9000310032002FB09700BFB097004FB197009E
:104CA000DFB1970027040700E00F5000E08F5800A5
:104CB000E00F5900E08F590027003A00E10F54003F
:104CC0002500340054692D0065822E00B6E02200D4
:104CD000170124005FA89700EFA897007FA997000D
:104CE0008FB19700080407000000E00002003D00BB
:104CF00069045400010037006804540098AF9F0015
:104D00001FA89700AFFD07000002BE000203BE000F
:104D1000D4AF9F00E5AF9F00F6AF9F0087B79F001D
:104D20002FB09700BFB097004FB19700DFB1970049
:104D30008AFB0700030407000004BE006000B800FF
:104D40006011B800A0B79F00B1B79F00C2B79F0025
:104D5000D3B79F00160037002FB09700BFB0970061
:104D60004FB19700DFB19700F60307000004BE00C3
:104D7000250407000002BE000203BE002FB097000A
:104D8000BFB097004FB19700DFB197003D04070017
:104D90000002BE000203BE00A4B79F00B5B79F008B
:104DA000C6B79F00D7B79F000000EB0090AF9F00F1
:104DB000A1B4200010C0B30005003700E48040001B
:104DC000B10F5400A18F5C00030039000040E800DF
:104DD000EA4F5000F9FF3A00E0CF9F009FA89700EC
:104DE00081805500EFB29700858050000000FB00E5
:104DF000008550000500E000010032000A05E900CE
:104E000063006700010032000A05E9000E28A300D4
:104E100039003200610167000E18A3000F00320054
:104E20003C0090000068A30006003200B1022000A0
:104E30000200E000010032008180E8000D017800EE
:104E40000D003700B00220000200E0000100320037
:104E50000080E8008C0078000E0037000200E000BF
:104E6000220032003C0090000068A30007003200DE
:104E70000D017800010220000C007800B4FD07004D
:104E80000000E00006003A00180037008C007800AF
:104E9000000220009A020700E10F400013003200D8
:104EA0008D06E800110037003C0090000068A30068
:104EB000070032000D017800010320000C0078008B
:104EC000A3FD07000000E00006003A0006003700DE
:104ED0008C0078000003200089020700E10F4000E9
:104EE000010032008D06E8000A05E9000A00E00032
:104EF000EDFF3C00570037000E38A30014003A00C5
:104F0000110037003C0090000068A3000700320049
:104F10000D017800010220000C0078008CFD0700D4
:104F20000000E00006003A00060037008C00780020
:104F30000002200072020700E10F40000100320071
:104F40008D06E8000A05E9000A00E000EDFF3C00DC
:104F5000610167000E18A3000E0032003C009000B3
:104F60000068A30005003200B10220000200E0004A
:104F7000220032008180E80020003700B0022000CB
:104F80000200E000010032000080E8008C007800A0
:104F90002C0037000200E0002E0032003C009000A0
:104FA0000068A300030032000D0178000102200018
:104FB000130037008C007800000220002100370029
:104FC0003C019000A0B420008100FB000268A30017
:104FD00010003200C208DD00810040001101BE0057
:104FE0000800BE00F6FB0700A2002000030020001E
:104FF000A603070001032000808040000D01780017
:105000000C00780052FD07000000E00010003A009C
:1050100010003700C208DD00810040001101BE0011
:105020000800BE00E6FB0700A200200003002000ED
:105030009603070002032000000141008C00780065
:10504000020078002E020700E10F4000010032004C
:105050008D06E8006FC897008040E900E1CF9F000F
:105060000004E000D6FF3A00130037003C00900037
:105070000068A300070032000D0178000103200042
:105080000C00780032FD07000000E00006003A0046
:10509000060037008C00780000032000180207008B
:1050A000E10F4000010032008D06E8001FA89700C4
:1050B0000000E90090AF9F001FA897000000E000EB
:1050C000EAFF3C006FB39700E80F53000300340081
:1050D00080C0B300E0CF9F0002003700CFEB970005
:1050E000E7CF9F006FC897008005FB00EFB09700E7
:1050F0008B8550000004E000100032003C0090005E
:105100000068A300070032000D017800E1022000D2
:105110000C0078000EFD07000000E00006003A00D9
:10512000060037008C007800E0022000F401070040
:10513000E10F4000010032008D06E8006FC99700C2
:105140000200FB009FFC07000002BE000203BE003D
:105150002FB09700BFB097004FB19700DFB1970015
:1051600021FB0700F70207002D0037003C019000EB
:10517000A1B420000000FB000268A3001000320070
:105180004200DD00808040001101BE000800BE002A
:105190008BFB0700A2002000030020003B03070058
:1051A00001032000808040000D0178000C00780091
:1051B000E7FC07000000E00010003A001000370094
:1051C0004200DD00808040001101BE000800BE00EA
:1051D0007BFB0700A2002000030020002B03070038
:1051E00002032000000141008C00780002007800DA
:1051F000C3010700E10F4000010032008D06E80006
:10520000EFC997000300FB004200DD00A1B42000BD
:10521000008040001001BE000800BE001B03070014
:105220000004BE00EFC897000140E900E0CF9F00F6
:105230000104E000CDFF3A00110037003C0090006F
:105240000068A300070032000D0178000103200070
:105250000C007800BEFC07000000E00006003A00E9
:10526000060037008C00780000032000A40107002E
:10527000E10F4000010032008D06E8008B05E900D7
:105280000B00E000EDFF3A000E38A3009001320061
:105290000A00E0008E0134003C0090000068A3008A
:1052A000070032000D017800010220000C00780098
:1052B000A7FC07000000E00006003A0006003700E7
:1052C0008C007800000220008D010700E10F4000F3
:1052D000010032008D06E8000A05E900EEFF3A0001
:1052E0007B0137008E007800010CB20011003A00FB
:1052F0000000E000040032001FB297004404BE002A
:1053000094B79F00040037009FB2970045047800CF
:1053100095B79F00CFC4DE00E00F5400E08F5C0023
:105320000E003D003E00B30060041400E0841C0049
:105330000A0037000000E000040032001FB39700AD
:105340004604BE0096B79F00040037009FB3970045
:105350004704780097B79F008004EB006FB0970078
:105360000000E00006003A000880740000F0A7008A
:105370000000EA000000E9004F00DE00E0B79F00F7
:105380008E007800010CB200C1AF9F000004200025
:10539000808F50002300320003003C000100E00039
:1053A000080032002D003700000820004FA99700A8
:1053B000800F51000D003200000C2000800F5100C2
:1053C00026003A00A1B4200010C0B300E4804000E1
:1053D000B10F5400A18F5C001F0039000040E800AD
:1053E000EA4F5000F9FF3A001B00370010C0B3002D
:1053F0000201200003002000820F5400838F5C0014
:1054000015003900441ADD00CC11DE008301720062
:105410004411DD000040E800E84F5000F6FF3A007C
:105420000D00370010C0B3008200200003002000F0
:10543000820F5400838F5C0007003900C31ADD001F
:10544000CD11DE00838172004311DD000040E800D1
:10545000EB4F5000F6FF3A00E0CF9F006FCB970074
:105460000600FB00EFB39700870F500002003D00DD
:10547000E7CF9F0004003700EFB09700808F500007
:1054800001003D00E0B79F000B00E0000300320088
:1054900063006700010032008B05E9000EE8A300FD
:1054A000060032006FB19700828F55000200340071
:1054B00082855500010037008005EB00EFC9970099
:1054C0000300FB000002EB00A4B79F00808F550093
:1054D0000200340000805500A0B79F000E28A300F2
:1054E0003C003200610167000E18A3000F0032007B
:1054F0003C0090000068A30006003200B1022000CA
:105500000200E000010032008180E8000D01780017
:105510000D003700B00220000200E0000100320060
:105520000080E8008C0078000E0037000200E000E8
:10553000100032003C0090000068A3000700320019
:105540000D017800010220000C00780000FC07002B
:105550000000E00006003A00060037008C007800EA
:1055600000022000E6000700E10F400001003200C9
:105570008D06E800AFB297000500E000520032004F
:10558000050578003C0090000068A3000700320089
:105590000D017800010320000C007800ECFB0700EF
:1055A0000000E00006003A00060037008C0078009A
:1055B00000032000D2000700E10F4000010032008C
:1055C0008D06E8000A05E900EEFF3A00AAB79F0041
:1055D0003D0037002FB397000600E00016003200B0
:1055E0000E38A30014003A00060578003C00900035
:1055F0000068A300070032000D01780001022000BE
:105600000C007800D2FB07000000E00006003A0022
:10561000060037008C00780000022000B800070068
:10562000E10F4000010032008D06E8000A05E900A4
:10563000EEFF3A00AAB79F00610167000E18A300B1
:105640000F0032003C0090000068A300060032000A
:10565000B10220000200E000010032008180E80079
:105660000D0178000D003700B00220000200E000BC
:10567000010032000080E8008C0078000E00370046
:105680000200E000100032003C0090000068A3001F
:10569000070032000D017800010220000C007800A4
:1056A000ABFB07000000E00006003A0006003700F0
:1056B0008C0078000002200091000700E10F4000FC
:1056C000010032008D06E800EFB397000702E90001
:1056D0006320B90000017800A2AF9F004222DD00E4
:1056E000A0B420000002420004057800CFAD97006E
:1056F0005C003700EFB197008301E900E3B79F003A
:1057000000042000808F55003700320003003C0069
:105710000B00E000070032003D00370000082000C9
:10572000808F550020003200000C2000808F550033
:1057300037003A000E48A300100032001A02BE00E3
:105740000401BE000800BE00F4B79F0085BF9F00A3
:105750001BFA0700E0CF9F000000FB00CF80DE00B7
:105760007FB297008FBA97000401BE00CA010700FC
:105770000004540081845C00070037001A0178009F
:10578000110009000284D800A200200011000900C5
:105790000280D800E1CF9F006FCA97000443B00099
:1057A000E4CF9F001A00370010B320000E58A3006A
:1057B0000100320000B22000A1B420008100550099
:1057C0000801BE008100E900030033008301D1001D
:1057D0000281D300FBFF37006F0161006041790057
:1057E000E2CF9F000A0037000800BE00AFAA970072
:1057F0008502E900030033008100D1000080D3005E
:10580000FBFF3700674060000043B000E0CF9F001F
:10581000BC0090006FCB97000600FB000168A3005E
:10582000070032000D017800800078000C0078003D
:1058300047FB07000000E00005003A0005003700C4
:105840008C0078002E000700E10F400001003200BC
:105850008D06E800AFAB9700E3835300A7AF9F002E
:10586000640555006FB097000000E000A1FF3A000A
:105870000E38A30016003200AFB097000100E00020
:1058800013003400010578003C0090000068A3007C
:10589000070032000D017800010220000C007800A2
:1058A0002BFB07000000E00006003A00060037006E
:1058B0008C0078000002200011000700E10F40007A
:1058C000010032008D06E8000A05E900EEFF3A000B
:1058D0003FA9970012407800E0CF9F000004E0004D
:1058E00034FB3A000D0078004F0778004F06BE00E9
:1058F0004F05BE004F04BE006F02B100000006005D
:10590000889FBE0001047800B80090008084EB00FE
:105910000118A3003A003200180190000198A3007A
:1059200002003A000200E00035003A000190A000B9
:105930003104980080047800F90FB2000200E00002
:1059400002003A0028009000000C7800EA8F540012
:1059500005003A000178A30003003A0088007800AF
:10596000D0002000E6FF070018009000D80090004B
:10597000810F50000B0032000000E8001004980076
:105980001800780009487800000CE80011C0B30046
:1059900080BD200001487800EA8F540018003A00CA
:1059A00005003700880078000940780017000700DC
:1059B0008004780012003700380090000088A300AF
:1059C0000F00320018019000A800900048009000DD
:1059D0001FF8070098009000810F5000040032006B
:1059E000380090000003B300300498008084EB007E
:1059F0000000EB001004980028009000000C7800D4
:105A0000090078004F04BE00000006000200FA0002
:105A1000889FBE00A0FF9F0001047800380090001E
:105A20000068A30033003A00E200600005003A007D
:105A30000003B30030049800110498000080EB00CC
:105A40002E003700D80490000900E00006003A005C
:105A500012002000E680570048009000FCF7070085
:105A60001904980023003700A80090000100E0000E
:105A700008003A00B1BD200021049800010C780014
:105A80002100200051049800110498000030A0006B
:105A90003004980018019000A80090004800900081
:105AA000EBF70700280090008080EB0011049800BD
:105AB000AFF8970001487800000CE8002FF8970035
:105AC000EA4F50000B003A00380090000088A30015
:105AD0000800320018019000A800900048009000D3
:105AE000DBF707000000EB0010049800A80090000E
:105AF000010C7800AFF897000100FB004F04BE00D6
:105B00000080FA000000060000C0DA000000060075
:105B10002800FA00889FBE008A9FBE008C9FBE00AE
:105B200007067800878669000C003B0003047800B4
:105B30008704780008F0A10009F0A100840F50004C
:105B4000858F5800860F5900890F5C0003003300D1
:105B50000CF0A20001003A000CF0A10085F807004B
:105B60006400E1005F003200780147006408E10052
:105B7000610032006C014700748557003200BE009E
:105B80001201BE003A04BE001A05BE001E039000BA
:105B9000BE0A90008503530006003D000004FD008E
:105BA0008104FD000205FD008305FD008703EA0076
:105BB000050378000DF8A30004003200600414000F
:105BC000E0841C0060051D00E0851D006022B80017
:105BD0007D0320000D38E1008006EB000B0039004A
:105BE0004433DD00F300B200830173003900370055
:105BF000848272000D027800E10664008B85D1007A
:105C00000A85D3008984D3000884D3008703E90080
:105C1000F7FF3B0008004000898048000A01490066
:105C20008B81490004003B0060001000E0801800F8
:105C300060011900E08119000358A3000900320037
:105C40008D82720084827200610260008301D10043
:105C50000281D3008180D3000080D3000603E800D6
:105C60001B0037000348A30017003A000600E000BD
:105C7000170034000603E9000D00A30000004800EF
:105C80008180480002014900838149000348A30044
:105C90000F003A000600E000090034000603E900A6
:105CA00000004000818048000201490083814900D2
:105CB00001003A000003EB000348A300F5FF3200A7
:105CC0006022B800020037008482720061826600A0
:105CD000FCF7070003F0A1000CF0A70003F0A00000
:105CE00038F83700640147006408E10002003A0018
:105CF0000DF8A30030F83A003200BE001201BE00D9
:105D000030F83700000000008F1FD1006800070046
:105D10008F87E9000000E00000000600809FEB0094
:105D2000630007008F87E9000000E0000000060024
:105D3000801FEB005E0007008F87E9000000E00095
:105D4000000006001400FA00889FBE008A9FBE0073
:105D50008C9FBE000004BE000205BE006800470024
:105D60000A90BE000890BE00B3F807000070A700BC
:105D70000BF0A1000BF8A30020003A009E09900050
:105D80000E099000FE0090006E0090009E029000B0
:105D900034432000848252000AF832000A003C009A
:105DA000B4FC2F000428E100140034008301D1006A
:105DB0000281D3008180D3000080D3008502E800F7
:105DC000FAFF3A00FFF73700B40020000428E10092
:105DD00007003C00000040008180480002014900AB
:105DE000838149008502E900FAFF3A00F5F73700A0
:105DF0000300280002002000010037006011B800F5
:105E00006000B800EFF737006011B800C1F8370044
:105E10001400FA00889FBE008A9FBE008C9FBE00BF
:105E2000040678000004BE000205BE0068004700BA
:105E30000A90BE000890BE007FF807006200E100F3
:105E40000800BE000A01BE00040020000B003A005A
:105E50001E029000E43FB1006E009000FE00900032
:105E60000E0990009E099000F300B20005FE230089
:105E7000858171000BF0A70003F0A000040E7800EC
:105E8000D0F7370007F0A20021FF37004CF80700D9
:105E90000400BE0000000600020AB900001BB900A1
:105EA0000200B800810042008100430000000600AB
:105EB000889FBE008A9FBE008C9FBE000404BE0067
:105EC0000605BE00809FBE00829FBE002100070025
:105ED000040678000800BE000A01BE001D0007008D
:105EE000840678004F03BE004F02BE008D4F76003F
:105EF0007FB0970013003300F0FF2F008B8F6B00F3
:105F000006003B000D0666000C00A7000A003700E3
:105F100007F0A600100020000A003700880F52008A
:105F2000898F5A008A0F5B008B8F5B00030039005A
:105F30001000200001003E000000200007F0A70034
:105F40000000EA004F06BE004F05BE004F04BE0031
:105F50000000060005FF27000582610007003200EF
:105F60000428E100010032002400050006000700BB
:105F700001003A0044000500040805000200070083
:105F8000F9FF3A00140005006F8261008102700081
:105F9000850271008502720000000600B54D000008
:105FA0004F47000049320000205300006572000096
:105FB000696100006C0000002D2D00002D2D0000F7
:105FC0002D2D0000763200002E3000002D2D000017
:105FD0002D2D00002D2D000000760000322E000037
:105FE000302D00002D2D00002D2D00002D53000020
:105FF0004E3A0000253000003364000000F000003D
:1060000025300000327800003A25000030320000D0
:10601000783A0000253000003278000020DF0000D0
:10602000253300002E31000066B000000A50000049
:106030003A25000034690000204F00003A25000096
:1060400034690000002000004456000000500000A9
:106050006F740000693A0000202500002E32000015
:106060006C660000205600000D0A0000004F000082
:10607000707400006F3A0000202500002E320000EE
:106080006C660000205600000D0A0000000D0000A4
:106090000A410000757400006F6D0000617400001B
:1060A0006120000053630000616E0000204F00007B
:1060B000464600000D0A0000000D00000A410000E5
:1060C000757400006F6D00006174000061200000B5
:1060D00053630000616E0000204F00004E0D000071
:1060E0000A000000754D00006F6700006932000073
:1060F0000D0A00000052000054430000432000003D
:106100004F4B00000D0A0000003F00000D0A000088
:106110000000000012010000000200000200000068
:1061200000080000D80400000A0000000001000080
:10613000010200000001000009020000430000000D
:106140000201000000C0000032090000040000004D
:106150000001000002020000010000000524000010
:1061600000100000010400002402000002050000ED
:1061700024060000000100000524000001000000CA
:106180000107000005810000030A00000002000072
:106190000904000001000000020A000000000000E5
:1061A000000700000502000002400000000000009F
:1061B000070500008202000040000000000000000F
:1061C00004030000090400000A0300004D00000061
:1061D0004F000000470000004900000026030000B7
:1061E000550000004D0000004F0000004700000077
:1061F00049000000320000002000000053000000B1
:1062000065000000720000006900000061000000ED
:106210006C00000020000000700000006F00000013
:1062200072000000740000009CB00000E0B00000AC
:10623000E4B00000EEB00000020400000E01000017
:106240000F1100000F000000020400000E110000FA
:106250001F1000000E000000020400000C040000EB
:10626000040400000E000000020400000E110000F3
:10627000111100000E0000000204000011110000C6
:10628000111300000D0000000A00000011110000B1
:10629000111300000D000000050A0000111100009C
:1062A000111300000D000000050A00000E1100008F
:1062B000111100000E000000040A00000A0A00008C
:1062C000111F00000E000000000E00001517000056
:1062D000110E0000000000001C020000010500007B
:1062E000091E0000080400000200FA009EC0A90078
:1062F0000080EB00702488000080EB0050248800B0
:10630000AA24EF00420020008000EB00C04A2000D9
:10631000B2F707002000200030258800A824EF00F5
:106320008644A900F009200080248800F00920009C
:106330006024880082C4A8008804A80000C020004F
:106340004800DE00C02488000040EB00004F7800C9
:10635000070037001E80FB00C200DD0000C02000E7
:10636000008140006000B8000089BE001E4FE800B8
:106370001E407800EB4F5000F6FF36009424A80032
:106380009624EF0094A4A9009424A9008000200082
:106390005024880020B820008040EB00014878009D
:1063A00080B820008040EB0001487800415C80000C
:1063B000F00F200000806000405C8800515C80008D
:1063C00000F02F0000806000505C880050248000A6
:1063D000680060000000E000ECFF3A0010C0B3006D
:1063E00013E8B70010C0B30014E8B7001568EF0059
:1063F0001668EF000D68EF000040EB00004F7800DA
:10640000170037001E80FB0080004000A0B720006E
:10641000008040008000EB00010878001E80FB0037
:106420008000400040B72000008040008000EB006A
:10643000010878009E80FB00E0B82000008040004A
:106440008040EB00014878009E80FB0020B92000CE
:10645000008040008040EB00014878001E4FE800BB
:106460001E407800E24F5000E6FF360080C020005A
:10647000D05B8800D00020005025880050B9200053
:106480001060880000C0200081C0B300014878007F
:1064900010C0200041C0B3000148780010C02000A7
:1064A00010407800804078000174A00010C02000E7
:1064B000014878000268EF001828EF001A28EF0062
:1064C0001C68EF000028EF000080FA0000000600C2
:1064D0000200FA0000408000E10F50000B003A007B
:1064E000A124800000042000008060000000E00083
:1064F00006003A000080EB00502488008C04A800BD
:106500008C84A80020002000004088000024800027
:10651000700060000000E0000700320010248000DE
:10652000700060000000E000030032000001200065
:1065300000248800BD040700402480006200600041
:106540000000E000020032008EC0A900A100370068
:1065500050248000610060000000E0000A0032006A
:1065600060248000610060000000E000060032004E
:106570005DFF07009EC0A80040002000004088008A
:10658000100020005024880050248000700060001B
:106590000000E00005003200602480007000600010
:1065A0000000E00001003200930407000124800095
:1065B00000042000008060000000E00003003200C2
:1065C0000004200000248800F30607005024800007
:1065D000640060000000E0001400320060248000CD
:1065E000640060000000E00004003200120020009F
:1065F0008000EB0030072000FA1007004000200068
:106600005024880011C8BF000004E00003003200DD
:1066100011C8BF000040E90011E8B70011C8BF0071
:106620000004E00001003A00A301070051248000AB
:1066300000082000008060000000E000060032003A
:106640006124800000082000008060000000E0005D
:10665000010032004C0407005024800062006000FA
:106660000000E0000C003200602480006200600046
:106670000000E00008003200120020008000EB0063
:10668000F0FF2700D71007000080EB00702488007F
:10669000200020005024880000408000E30F5000BC
:1066A00002003E008EC0A9004A003700602480002E
:1066B000680060000000E000450032000040EB0090
:1066C000004F78003D0037005024800068006000D3
:1066D0000000E0003D00320090248000004078007F
:1066E0000EE8B7000EC8BF000080FB004400DE00CB
:1066F000004078000FE8B700800020005024880098
:106700000EC8BF00684060000004E00011003A00BD
:106710000FC8BF000081FB008080FB0020B9200073
:10672000008040009040780061C060000004A2003A
:10673000E140600020B9200000004100E1C060009D
:10674000104178000204A1008140710001487800E6
:10675000100037000FC8BF000081FB008080FB00E5
:10676000E0B82000008040009040780061C06000E8
:106770000004A200E1406000E0B8200000004100F9
:10678000E1C06000104178000204A1008140710066
:10679000014878000FC8BF000004E00002003A0082
:1067A0002E040700040037000001EB00E180200008
:1067B000200720008B1007001E4FE8001E407800C5
:1067C000E34F5000C0FF360001003700000000001A
:1067D0008EC0A9000080FA00000006000400FA0044
:1067E00020479800314798003E4090000080FB0011
:1067F000680060000000E000030032008040EB0011
:106800002E4090009B0107003E4090000080FB005E
:10681000640060000000E0000300320011C0B3001B
:106820002E40900093010700A14A20002E409000C6
:106830000080FB0000004000008F40001E00780038
:10684000BE409000014878000080FA000000060079
:106850000800FA0020479800314798002207980066
:10686000634798003E4090000004E00007003200BB
:106870002E4090000080FB0080004000A0B7200068
:1068800000804000100F7800060037002E40900076
:106890000080FB008000400040B7200000804000E6
:1068A000100F78001E0078000000E00002003A009F
:1068B0000000EB0037003700AE0090001E007800AB
:1068C000110098001E007800EE409000014878000A
:1068D0001E0078001040900002C4B30082406000A7
:1068E0001E007800114098001E00780010409000B3
:1068F000804078000134A0001E007800114098000C
:106900001E00780010409000804078000174A000C4
:106910001E007800114098003E4090000004E00006
:106920000E0032002E4090000080FB00AE40900030
:106930008180FB0001814000A1B72000810041005F
:10694000910078000120A20000014000A0B72000C3
:1069500000004100010878000D0037002E40900033
:106960000080FB00AE4090008180FB000181400070
:1069700041B7200081004100910078000120A20071
:106980000001400040B720000000410001087800ED
:106990001E0078000080FA00000006000400FA00E3
:1069A00020479800314798002E4090000004E000F6
:1069B00017003A003040800081C0B30001487800E1
:1069C0003040800051B92000110098003040800014
:1069D000C1C0B300114098003040800031408000B9
:1069E000914090000174A00011409800D05B80009D
:1069F00041C0B30011409800D05B8000D15B8000A3
:106A0000914090000174A000114098002E003700C2
:106A10002E4090000080FB000000400080007800C5
:106A20003E4090000080FB00008040004300DD00FD
:106A30008000780000C02000008F40001E00780019
:106A400010409000804078000124A0001E007800D3
:106A5000114098001E00780010409000804078009F
:106A60000174A0001E007800114098002E40900094
:106A70000080FB0000004000800078003E40900055
:106A80000080FB00008040004300DD00E400400087
:106A900000C02000008F40001E00780010409000D1
:106AA000804078000124A0001E007800114098006A
:106AB0001E00780010409000804078000174A00013
:106AC0001E007800114098000080FA0000000600C7
:106AD0000200FA00004F7800A1248000000220008C
:106AE000008060000000E000510032001E80FB00CA
:106AF00080004000A0B72000008040001002780015
:106B00001E80FB0080004000A0B7200000804000F5
:106B1000100078001001BE000004200001002000D9
:106B2000820278000301780080017800010078007B
:106B300083826200000061008000EB00C000DD0085
:106B4000000020000001BE006128B80000017100B3
:106B500081817100028ABE001E80FB00800040001F
:106B6000A0B7200000804000100278001E80FB00CB
:106B700080004000A0B72000008040001000780096
:106B80001001BE0000042000010020000000690088
:106B900081806900008ABE001E80FB009E80FB0091
:106BA00001814000A1B720008100410091007800E0
:106BB0000120A20000014000A0B720000000410019
:106BC000010878001E80FB0080004000A0B7200074
:106BD00000804000900078001E80FB000001400013
:106BE000A0B7200000004100100078001040900085
:106BF0000044B200904098001E80FB0080004000DE
:106C0000A0B7200000804000900078001E80FB00AC
:106C100000014000A0B720000000410010007800F3
:106C20001041900000C4B3000040690090409800FB
:106C30000080FA00000006000000FA009424EF0033
:106C40008C24EF000028EF000080FA00000006000E
:106C50000000FA00004080000000E00014003A004C
:106C60009424EF008C24EF002000200030258800C1
:106C7000A824EF008644A900F009200080248800A1
:106C8000F00920006024880082C4A8009EC0A800EB
:106C9000010037009404A800A02480006100600077
:106CA0000000E000FBFF32001000200000408800E0
:106CB0000080FA00000006000000FA0013C8BF00C0
:106CC0000004A2000004E0003400320010C0B30051
:106CD00013E8B70014C8BF000004A2000004E000DD
:106CE0002E00320010C0B30014E8B70009C8BF007E
:106CF000E24F50000C003A00D05B80008040EB0077
:106D000001487800D05B800081C4B3001140980036
:106D1000D05B8000D15B8000914090000174A000A6
:106D2000114098001D00370009C8BF00E14F500016
:106D30001A003A001068EF002040800081C0B300C4
:106D4000014878002040800051B9200011009800CF
:106D50002040800041C0B3001140980020408000D6
:106D600021408000914090000174A00011409800E3
:106D700010C0B30010E8B7003040800081C0B300FD
:106D8000014878003040800051B92000110098007F
:106D90003040800001C8B300114098000080FA0024
:106DA000000006000000FA001568EF001668EF000A
:106DB00009C8BF00E24F50000F003A003040800089
:106DC00081C0B3000148780030408000E1B9200064
:106DD000110098003040800081C4B3001140980039
:106DE0003040800031408000914090000174A0004C
:106DF000114098001D003700B0B920001080FB0042
:106E0000C1B920009180FB00C808DD0001007000BE
:106E100080007800205C8000808F500007003100E7
:106E2000B0B920001080FB00C1B920009180FB00A8
:106E3000C808DD0001007000205C88009600070093
:106E4000D05B8000E1B9200011009800D05B800089
:106E500081C4B30011409800D05B8000D15B8000FA
:106E6000914090000174A000114098000080FA0049
:106E7000000006000400FA002047980031479800FF
:106E800000C02000000F78002E4090000080FB0022
:106E900000004000800078003E4090000080FB0031
:106EA000008040004300DD001E0F40001E007800FF
:106EB0009000780001F0A100010878003E409000A9
:106EC0000004E00007003A002E4090000080FB0024
:106ED0008000400040B72000008040001E0878007D
:106EE000060037002E4090000080FB00800040002C
:106EF000A0B72000008040001E0878001E00780027
:106F00009000780001E0A100010878009E00780060
:106F1000648040009000780001E0A0000108780043
:106F20000080FA00000006000000FA0094A4A90006
:106F3000115C800000082000008060000000E0007C
:106F400027003A0080B820009040780000C8B300C5
:106F500000C060000004E0000A00320020C0B3005E
:106F600009E8B70016C8BF000004A2000004E00052
:106F7000010032008BFF07001468EF001368EF0078
:106F8000430037003040800081C0B30001487800E2
:106F90003040800051B9200011009800304080003E
:106FA000C1C0B300114098003040800031408000E3
:106FB000914090000174A00011409800D05B8000C7
:106FC00041C0B30011409800D05B8000D15B8000CD
:106FD000914090000174A000114098002C003700EF
:106FE00050B920009040780000C8B30000C0600095
:106FF0000004E0000F00320010C0B30009E8B70041
:1070000015C8BF000004A2000004E0000100320027
:1070100064FF07001468EF001368EF0012C8BF0098
:107020000004A2000004E0001900320022FF070063
:107030001700370020C0B30009E8B70030408000D7
:1070400081C0B300014878003040800051B9200071
:10705000110098003040800041C0B30011409800FA
:107060003040800031408000914090000174A000C9
:10707000114098001468EF001368EF0012C8BF00B9
:107080000004A2000004E000010032000AFF070033
:107090000080FA00000006000200FA0080C0B30081
:1070A000004F7800205C8000E70F50000D003E008C
:1070B000205C8000004F780008C8BF000004E0009A
:1070C00003003A0010C0B30008E8B700050037001D
:1070D00008C8BF00E14F500002003A0020C0B300D2
:1070E00008E8B700215C80001E80FB000080500093
:1070F000205C8800D05B80001E487800E0B920004A
:1071000050408800105C8000610060000000E000DA
:1071100017003A000900370051408000005C8000F1
:1071200010417800824878008100E80051408800D2
:107130000000E800005C88001E4FE9001E40780057
:107140000004E000F4FF3A000C00370051408000DA
:10715000005C800010417800824878008100E800DF
:10716000514088000000E800005C88001E4FE900E4
:107170001E4078000004E000F4FF3A000080FA00AE
:10718000000006000200FA0020408000104F780046
:107190009E80FB00405C80004800DE00535C800065
:1071A000F20F2000028161004811DD000200700032
:1071B000808F500008003600405C80004800DE00F0
:1071C000525C8000F10F200081006100C808DD00E2
:1071D00001007000004F7800405C80004800DE0035
:1071E000525C8000F10F200081006100C808DD00C2
:1071F00001007000800078001E80FB0000805000BD
:10720000F10F200081006000C808DD00435C8000B1
:10721000F20F20000281610082807000415C8800D2
:10722000C800DE00F00F200000806000525C80008B
:1072300001F02F008100610001007000505C8800A7
:107240000040EB00104798000C003700305C8000D5
:107250009E4090000181FB00E1B9200081004100C7
:1072600091407800014878000000E800305C880018
:107270001E4090000040E800104798001E4090001B
:107280009E4F5000F1FF3900405C80004800DE0056
:10729000525C8000F10F200081006100C808DD0011
:1072A000010070000000E0001E003200304080004D
:1072B00081C0B3000148780030408000E1B920006F
:1072C0001100980020408000900078000000240009
:1072D000008060000000E00009003A0030408000BB
:1072E00081C4B300114098003040800031408000DC
:1072F000914090000174A0001140980030003700C8
:107300003040800081C0B3001140980030408000C0
:1073100031408000914090000174A000114098001D
:10732000270037003040800081C0B300014878005A
:107330003040800051B9200011009800304080009A
:1073400041C0B300114098003040800031408000BF
:10735000914090000174A00011409800505C8000A2
:107360004800DE00625C8000F10F200081006100B7
:10737000C808DD00010070000000E00008003200D5
:10738000505C80004800DE00625C8000F10F20004D
:1073900081006100C808DD000100700000000100EC
:1073A000405C80000070A100405C880012C8BF00F3
:1073B0000004A2000004E000010032003EFE0700CD
:1073C0000080FA00000006000200FA00105C800055
:1073D0000070A000105C8800420020008000EB00DC
:1073E000C04A20007DF30700020320008000EB006C
:1073F00000C0200079F307009424A8000040EB00AF
:10740000004F78000B0037009E80FB00E0B82000A2
:10741000008040008040EB00014878009E80FB0027
:1074200020B92000008040008040EB000148780037
:107430001E4FE8001E407800E24F5000F2FF360079
:10744000220020008000EB0020B7200063F307003B
:107450009424A90080C02000D05B880000C02000D8
:1074600020408800204080003040880070B9200013
:107470001040780002E8B70002C8BF000004E00036
:1074800003003A0000012000004088000600370099
:10749000120020002180200010002000510D070064
:1074A00000022000004088000080FA000000060072
:1074B0000000FA0050B920009040780000C8B300E6
:1074C00080CF500047003A0020B8200001CCB30024
:1074D0000148780080B92000104078000080FB004F
:1074E000E20F500009003200E30F50002300320089
:1074F000E10F500037003A00A0082B00005C880024
:1075000020012000205C88003600370070B9200080
:10751000104078000004E00014003A0070B9200028
:10752000104078000080FB000000400080007800E0
:1075300040112B000080400010007800005C8800A3
:10754000005C80000080E8009040780040B8200097
:1075500001487800005C80006300400090407800A3
:1075600050B82000014878001E00370020B82000E5
:107570008040EB00014878001A00370070B9200005
:1075800010407800E24F50000E003E0070B920001D
:10759000104078000080FB00000040008000780070
:1075A00060112B000080400010007800005C880013
:1075B000005C8000104078000080FB00205C8800A8
:1075C0000800370020B820008040EB000148780018
:1075D0000400370020B820008040EB00014878000C
:1075E000000000000080FA00000006000200FA001F
:1075F000E0B920008040EB0001487800F0B920009D
:107600008040EB000148780050B92000904078009D
:107610007FC060000080FB00E10F500011003200CD
:10762000E20F5000130032000000E00047003A0073
:10763000105C80000070A000105C88000CC8BF00C7
:107640000004E0003A003200E0B920001040780069
:10765000804078000114A000E0B9200001487800C3
:107660003A003700105C80000070A000105C8800B9
:1076700036003700105C80000070A000105C8800AD
:1076800090B92000104078006F4060000004E000D6
:107690002900320090B920009040780000C8B30063
:1076A00000C060000004E00009003A0090B920002A
:1076B000904078006FC060000080FB0080004000B8
:1076C00040B7200000804000100F7800080037000D
:1076D00090B92000904078006FC060000080FB00EF
:1076E00080004000A0B7200000804000100F78000C
:1076F0001E007800900078000000280000806000E4
:107700000000E0000E0032001E00780090007800BB
:1077100000402000008060000000E0000A0032000D
:10772000E0B9200011C0B30001487800070037001D
:1077300000000000050037000000000003003700D3
:10774000000000000100370000000000115C800014
:1077500000082000008060000000E0000800320007
:10776000E0B92000005C8800105C80000000A000F0
:10777000105C880040B8200021C0B30001487800A8
:107780000080FA00000006000000FA00502580008A
:10779000620060000000E000130032002040800022
:1077A0009040900000C8B30080CF50000D003A0018
:1077B000D05B80009040900040C8B30080CF500064
:1077C00008003A0020408000C1C0B300114098007A
:1077D0002040800021408000914090000174A00072
:1077E00011409800AA24A900000820005024880015
:1077F0000080FA00000006000000FA008284A80061
:10780000000120005024880010C0B3000DE8B7002C
:107810001C68EF000001EB008000EB005007200027
:10782000700C07000080FA00000006000000FA005B
:107830000D68EF000001EB008000EB004007200026
:10784000680C07008284A900000120000024880041
:107850001C68EF000080FA00000006000000FA003B
:10786000D0C2B30011E8B7000EC8BF000080FB0013
:107870000020A1000000E0001F003A000EC8BF0079
:107880000080FB004200DE00004078000080FB002A
:10789000C200DD0000C020000080400020408800C1
:1078A0002040800030408800304080000020A2004E
:1078B00030408800204080009000780000C0230005
:1078C0008080600000402300808F500008003A0054
:1078D000204080001000900082002000800078008E
:1078E00050B9200036F207000B00070008003700EF
:1078F0003D000700060037000EC8BF000080FB00F7
:107900000020A100E80F500001003A0053000700DA
:107910000080FA00000006000000FA000868EF008E
:107920001268EF001568EF001668EF001068EF00AE
:107930000968EF00D05B8000D15B8000914090002F
:107940000174A10011409800D05B80000020A200CB
:10795000D05B8800D05B8000D15B800091409000BC
:107960000174A10011409800D05B80000020A200AB
:10797000D05B880030408000314080009140900012
:107980000174A1001140980020B820008040EB0055
:10799000014878000000EB00205C880080B82000DF
:1079A0008040EB0001487800415C8000F00F20002F
:1079B00000806000405C8800515C800000F02F0077
:1079C00000806000505C8800830007000001EB002D
:1079D0008000EB0030002000020C070052FD070081
:1079E0000080FA00000006000000FA0009C8BF008D
:1079F000E24F500002003A00E2FD07001500370098
:107A00000968EF0010C8BF000004A2000004E000F5
:107A10000F0032003040800081C0B3000148780080
:107A20003040800051B920001100980030408000A3
:107A3000C1C0B30011409800304080003140800048
:107A4000914090000174A00011409800010037009F
:107A50001068EF000080FA00000006000200FA0043
:107A6000D05B8000100078004E00DE0061406000B6
:107A7000004F7800D05B80000020A200D05B88001F
:107A800000408000E80F50000E003A0070B920005E
:107A9000104078008080FB00F0072000008060002C
:107AA000B0248800B02480000000E0000300320011
:107AB0000001200000408800020037004000200044
:107AC0000040880009C8BF00E14F500025003A007F
:107AD000D05B8000E1B92000110098006EFD070026
:107AE00008C8BF00E24F500009003A00D05B800098
:107AF00041C0B30011409800D05B8000D15B800092
:107B0000914090000174A0001140980030003700AF
:107B10001E4078000004E00009003A00D05B8000BD
:107B200081C4B30011409800D05B8000D15B80001D
:107B3000914090000174A00011409800240037008B
:107B4000D05B800081C0B30011409800D05B800002
:107B5000D15B8000914090000174A000114098001A
:107B60001B00370080B820009040780000C8B300A8
:107B700000C060000004E00014003200505C80008F
:107B80004800DE00625C8000F10F2000810061008F
:107B9000C808DD00010070000000E00008003200AD
:107BA000505C80004800DE00625C8000F10F200025
:107BB00081006100C808DD000100700000000100C4
:107BC000405C80000070A100405C88000968EF0004
:107BD0000080FA00000006000000FA0050B9200002
:107BE000104078000046B2000004E00051003A0066
:107BF00060B92000104078000080FB00CF80DE00DC
:107C0000B200200003002000820F5000838F580034
:107C10004A003E00006001002100370022003700CA
:107C200048003700200037004600370006003700C4
:107C30000B0037003A0037000D0037000A0037000C
:107C40001B0037002A003700105C80000070A00085
:107C5000105C880080002000004088003A00370057
:107C600013FE070038003700D7FD07003600370045
:107C700020802000005C8800105C80000000A000D4
:107C8000105C880040B8200011C0B30001487800A3
:107C9000105C80000070A000105C88002A00370093
:107CA00052FE070028003700290007002600370091
:107CB00090B92000104078008080FB0020B72000A1
:107CC00000804000005C8800105C80000000A00084
:107CD000105C880040B8200011C0B3000148780053
:107CE000105C80000070A000105C88001600370057
:107CF000105C80000070A000105C880090B920002B
:107D0000104078000081FB0070B92000904078009E
:107D100020B7200000004100014878000A00370029
:107D20000001EB008000EB00200020002D0B07007D
:107D300005003700000000000300370000000000CD
:107D400001003700000000000080FA00000006007B
:107D50000600FA0070B9200010407800E14F500092
:107D600010003A0050B92000104078007F406000B9
:107D70000004E0000B003A00105C80000070A000DE
:107D8000105C880060B9200010407800E34F50007C
:107D900003003A0010C0B3000CE8B7000100370040
:107DA0000C68EF0070B92000104078000004E0007B
:107DB000F7003A0050B92000104078007F40600082
:107DC000E24F5000F2003A0090B9200010407800D5
:107DD0006F4060000004E000ED00320090B9200028
:107DE000904078006FC060000080FB00E20F500000
:107DF000E7003C000140800000022000808F50001E
:107E0000E3003A00105C80000070A000105C880065
:107E100090B920009040780000C8B30000C0600016
:107E20000004E00011003A0090B9200010417800F1
:107E30006F4061000080FB008000400040B72000E0
:107E400000804000100F780090B92000904078002A
:107E50006FC060008080FB0020B9200000804000DF
:107E600010407800404798001000370090B920007B
:107E7000104178006F4061000080FB0080004000EE
:107E8000A0B7200000804000100F780090B92000BB
:107E9000904078006FC060008080FB00E0B8200058
:107EA0000080400010407800404798004E4090000D
:107EB000614060000004E00004003A001E00780009
:107EC0000020A100000F7800030037001E0078009A
:107ED0000020A000000F780090B9200090407800AA
:107EE00000C8B30000C060000004E0000A003A00CF
:107EF00090B92000104178006F4061000080FB00C5
:107F00009E0078000001400040B7200000004100C2
:107F1000010878000900370090B9200090407800EF
:107F20006FC060000080FB009E00780000014000F0
:107F3000A0B72000000041000108780060B92000CF
:107F400010407800E34F50002C003A001E007800EB
:107F50009000780000002800008060000000E00031
:107F60001900320090B920009040780000C8B3009A
:107F700000C060000004E0000A003A0090B9200050
:107F8000104178006F4061008080FB0020B9200024
:107F900000804000904078000114A0000148780063
:107FA0000900370090B92000904078006FC0600051
:107FB0008080FB00E0B82000008040009040780006
:107FC0000114A000014878001E00780010409000C5
:107FD000804078000124A0001E0078001140980025
:107FE0001E00780010409000804078000174A000CE
:107FF0001E00780011409800650037001E007800D0
:108000000020A200000F78001E0078009000780089
:1080100000002800008060000000E0001100320035
:108020001E00780010409000804078000174A1008C
:108030001E007800114098001E007800104090004B
:10804000804078000164A0001E0078001140980074
:10805000220020009E00780050002000610A0700E6
:10806000060037001E007800104090008040780025
:108070000164A0001E007800114098001E007800E6
:108080000020A200000F78004E4090006240600087
:108090000004E00006003A001E007800900078001E
:1080A00000002800008060000000E0002400320092
:1080B00090B920009040780000C8B30000C0600074
:1080C0000004E0000A003A0090B920001041780056
:1080D0006F4061008080FB0020B9200000804000DC
:1080E000904078000114A100014878000900370091
:1080F00090B92000904078006FC060008080FB0045
:10810000E0B8200000804000904078000114A100F9
:10811000014878001E00780010409000B2C3B30000
:10812000824060001E00780011409800220020006C
:108130009E007800500020002A0A07000600370041
:108140001E00780010409000B2C3B300824060006F
:108150001E00780011409800A14A200090B920002C
:10816000104178006F4061000080FB00000040007B
:1081700000804000100798001E009000104078001A
:10818000804078000114A1001E0090000148780092
:108190000080FA00000006000000FA00C0408000E5
:1081A000D140800061004000E0804800C04088006D
:1081B000D14088000DC8BF000004A2000004E00008
:1081C000080032001CC8BF000040E8001CE8B700EF
:1081D0001CC8BF000004E00002003A0000C0EB0031
:1081E0001CE8B7000080FA00000006000400FA0056
:1081F000C2408000D3408000028FBE00C04080009B
:10820000D14080001E01BE00800F5100818F5900B7
:10821000F7FF3A001E00BE000080FA0000000600D2
:108220000000FA00F0FC2F0060198800111980008E
:10823000F0FF2100008060001019880025E3A900EC
:1082400010C0B30024E3B7002119800000F0210022
:1082500001007000201988002043A9000119800046
:10826000000E2000010070000019880021E3A80022
:108270004119800000FE2F00008060000020A00057
:10828000401988000080FA00000006000200FA0091
:10829000000F78001E007800004078007F406000EA
:1082A0000080FB007F0060004219800001FE2F006B
:1082B0008100610001007000401988002023A8009F
:1082C0000000000000198000610060000000E00074
:1082D000FCFF3200001880000080FA000000060059
:1082E0000000FA008460A90021058000F0FF28004A
:1082F0000080600000E0A000200588009460A800D5
:108300000021EF0000002200100888002000280053
:10831000200888000080FA00000006000200FA0031
:10832000000F78009021EF009221EF00810C800077
:1083300000C0210001007000800C8800900C8000BB
:10834000F001B300900C880000402000A00C8800D1
:108350001E007800B00C8800810C800080FF2F0088
:10836000008060006000B300800C88000080FA008C
:10837000000006000200FA00000F78001E007800DE
:10838000B00C88000080FA00000006000200FA002D
:10839000213A8000F0F32F0000806000203A88002E
:1083A0000100370000000000113A800000022000A8
:1083B000008060000000E000FAFF320040A7A90042
:1083C000103A8000000178000210A0006004200034
:1083D00071052000237420008049780081497800CD
:1083E00082497800113A8000F00B20000081600083
:1083F000600420007105200023742000804978006B
:1084000081497800824978007136800000FC2F0095
:10841000008060002001B300703688004135800084
:1084200000FC2F0000806000E001B30040358800B0
:108430008136800000FC2F00008060007000B300D7
:108440008036880071368000F00F2C0000806000BC
:1084500000B0A00070368800103A8000000178005B
:108460000260A00060042000710520002374200039
:108470008049780081497800824978000000EB004B
:108480009909070098F70700F1F90700F0C2A90061
:10849000F0E2A900F102A900F122A900D9E2A900A5
:1084A000E882A900E8A2A900D022A800D062A80012
:1084B000E102A800E122A800C902A900C922A9007E
:1084C000C9C2A900CD02A800CD22A9002C06070030
:1084D0001C070700E0FC2A008206070007080700C7
:1084E0000010270021002000710907000053270019
:1084F0003D080700004F78008040EB0000CCB3003F
:10850000410607001E407800E14F400003003A009A
:10851000C0FD2A0073060700090037001E80FB001B
:10852000801F7800D0FE2A00801F780080A22000E3
:1085300031EF0700E487570080A22000690607009A
:1085400000802400811E2000590907001B08070035
:1085500002402200430F2000001920007C03070086
:10856000C0538000D1538000E2538000F353800059
:10857000880807002AFF070059FF07008041800094
:1085800066FF070069000700901680006200600027
:1085900000F0A7000000EA000000E9004F00DE0044
:1085A000004078000080FB00610060004600DD00B4
:1085B000A11780000160A10001007000A0178800D1
:1085C000901680006800600000F0A7000000EA003C
:1085D0000000E9004F00DE00004078000080FB0052
:1085E000610060004700DD00A11780000170A1005C
:1085F00001007000A01788001117800000102000F3
:108600000080600000F0A7000000EA000000E90020
:108610004F00DE00004078000080FB006100600039
:108620004800DD00A11780000180A100010070005A
:10863000A017880011178000002020000080600033
:1086400000F0A7000000EA000000E9004F00DE0093
:10865000004078000080FB00610060004900DD0000
:10866000A11780000190A10001007000A0178800F0
:1086700011178000002020000080600000F0A7009B
:108680000000EA000000EA004F00DE000040780031
:108690000080FB00610060004800DD006116800082
:1086A0000180A10001007000601688001117800091
:1086B000002020000080600000F0A7000000EA0019
:1086C0000000E9004F00DE00004078000080FB0061
:1086D000610060004900DD00611680000190A1008A
:1086E0000100700060168800A6FF37000000FA0045
:1086F000A0B020008040EB0001487800C0B020000E
:1087000081C0B30001487800B0B020008040EB0089
:1087100001487800005822000100200030588800ED
:10872000415888000080FA00000006000200FA00AC
:1087300000408000FF0F50003901360040248000C7
:10874000620060000000E00037013A001FC8BF006F
:108750000004E00030013A0001C4B300809A200018
:10876000F4010700004F78001E4078000004E0008C
:1087700029013200020420008000EB00809E2000CE
:1087800096EE0700809A2000104078000080FB00E1
:108790006101B90060FF2F00F1FF2F0002004000CF
:1087A00083804800A206200003002000820F5000B2
:1087B000838F580010013E00006001001301370054
:1087C0000D0137000C013700100137000A01370096
:1087D000090137000801370007013700060137009B
:1087E000050137000401370003013700020137009B
:1087F0000101370000013700FF003700FE0037009D
:10880000FD003700FC003700FB003700FA0037009E
:10881000F900370060003700F7003700F600370036
:10882000F5003700F4003700F3003700F20037009E
:10883000F1003700F0003700EF003700EE0037009E
:10884000ED003700EC003700EB003700EA0037009E
:10885000E9003700E8003700E7003700E60037009E
:10886000E5003700E4003700E3003700E20037009E
:10887000E1003700E0003700DF003700DE0037009E
:10888000DD003700DC003700DB003700DA0037009E
:1088900085003700D8003700D70037003A0037008E
:1088A000D5003700D4003700D3003700D20037009E
:1088B00031003700D0003700CF003700CE0037003E
:1088C000CD003700CC003700CB003700CA0037009E
:1088D000C9003700C8003700C70037002200370042
:1088E000C5003700B2003700C3003700C2003700B0
:1088F000C1003700C0003700BF003700BE0037009E
:10890000BD003700BC003700BB003700BA0037009D
:10891000B9003700B8003700B70037001C00370037
:10892000B5003700B4003700B3003700B20037009D
:1089300013003700B0003700AF003700AE0037003B
:10894000AD003700AC003700AB003700AA0037009D
:108950002D00370014003700A7003700040037004F
:108960004100370055003700DDE2A800A8003700BD
:10897000DDE2A900A6003700EC82A800A4003700C1
:10898000EC82A900A2003700ECA2A800A0003700EA
:10899000ECA2A9009E003700DDE2A900EC82A9004C
:1089A000ECA2A9009A0037004000200037FE070023
:1089B0008041880080418000CF80DE0006ED070006
:1089C0006022B800060020000709240063EC0700BD
:1089D000646626006566260066662600A7002400F9
:1089E00001ED0700849E2000809FBE00829FBE0094
:1089F00070022B00801F780004007800FEED070055
:108A0000EA87570082003700500020001FFE070051
:108A10008041880080418000CF80DE00EEEC0700BE
:108A20006022B80006002000070924004BEC070074
:108A3000646626006566260066662600A700240098
:108A4000E9EC0700849E2000809FBE00829FBE004C
:108A500070032B00801F780004007800E6ED07000B
:108A6000EA8757006A003700E0418000E10F5000BC
:108A700006003A003C28EF00809E200062012000A2
:108A800071042B00CEED07006100370010002000BC
:108A9000E0418800809E200052012000D1052B007B
:108AA000C7ED07005A003700809E2000920020008A
:108AB00021072B00C2ED070055003700909A2000D7
:108AC0009040780000CDB30080C0400040002000FE
:108AD0008008DD00C0A7200001487800C0A7200062
:108AE00090407800A09A20001040780080C040009C
:108AF00000CDB30080C04000C0A72000014878002E
:108B0000B09A20009040780000CDB30080C04000B3
:108B1000400020008008DD00D0A720000148780038
:108B2000D0A7200090407800C09A20001040780024
:108B300080C0400000CDB30080C04000D0A720001E
:108B400001487800D09A20009040780000CDB30012
:108B500080C04000400020008008DD00E0A7200029
:108B600001487800E0A7200090407800E09A2000BB
:108B70001040780080C0400000CDB30080C04000AD
:108B8000E0A7200001487800C0538000D153800046
:108B9000E2538000F3538000FE060700809E200011
:108BA000A2002000B1072B0085ED07001800370058
:108BB000909A200090407800C0A7200001487800DB
:108BC000A09A200090407800D0A7200001487800AB
:108BD000B09A200090407800E0A72000014878007B
:108BE000C0538000D1538000E2538000F3538000D3
:108BF000E806070006003700809E200042002000A3
:108C000051082B006EED0700010037000000000046
:108C1000809E20000C0107005C0107000300370064
:108C20000000000001003700000000000080FA0092
:108C3000000006000000FA0050B920001040780043
:108C40007F406000E14F500078003A0050B92000AA
:108C50001040780002C6B3008240600000C2B3003A
:108C600080CF500073003A0090B920001040780087
:108C70000004E0000400320090B9200010407800A9
:108C8000E14F50006D003A0060B9200010407800BC
:108C90000080FB0001022000810F50002000320004
:108CA00001022000810F500005003C000000E000A0
:108CB0000A003200E10F500013003200600037005C
:108CC00011022000810F50004300320021022000D9
:108CD000810F5000480032005900370080B1200059
:108CE000005C880080002000205C8800105C800010
:108CF0000000A000105C8800105C80000070A000E4
:108D0000105C88004E00370080B12000005C8800B5
:108D1000105C80000070A000105C880048003700E4
:108D2000B0B920001080FB00C1B920009180FB0089
:108D3000C808DD0001007000F10F20000101600093
:108D400091B8200091417800E0C1610002C171003A
:108D500082487800C800DE00A0B8200010417800EA
:108D600060416100814071000148780060B02000DE
:108D7000F10F20000101600061B8200091417800EE
:108D8000E0C1610002C1710082487800C800DE00C5
:108D900070B820001041780060416100814071008E
:108DA00001487800B0B8200090407800E0C0600032
:108DB00001487800C0B8200090407800E0C0600012
:108DC0000148780080B82000904078000174A0002D
:108DD000014878001A00370060B02000005C88006D
:108DE00070002000205C880020B8200011CCB30067
:108DF000014878001200370070B920001080FB0095
:108E000081B920009180FB00C808DD0001007000DE
:108E1000004078002AE8B700105C80000070A000D5
:108E2000105C880000000000050037000000000012
:108E300003003700000000000100370000000000C0
:108E40000080FA00000006000000FA0000B02400D4
:108E5000010020003058880041588800A0B0200050
:108E60008040EB0001487800B0B020008040EB006B
:108E700001487800C0B0200081C0B30001487800EC
:108E80001E68EF0051C1B30010C0B30053F60700D5
:108E9000D1C1B30020C0B30050F6070003C4B30033
:108EA00062AC20008040EB0020C0B30068F60700F1
:108EB000304188002828EF001F68EF000080FA008A
:108EC000000006000600FA00000F78001107980065
:108ED000220798001E007800E50F500012003A00AB
:108EE000304180009E009000808F500006003A00C4
:108EF00003C4B30062AC20008040EB0020C0B3008C
:108F000053F6070030418800404180009E009000E9
:108F1000808F500002003A001F68EF002468EF00C5
:108F200010C0B300010037000040EB000080FA00E1
:108F3000000006000400FA00000F780021479800A6
:108F40001E68EF00304180000000E00006003200A3
:108F50003041800090007800000028000080600010
:108F60000000E00022003A0030418000904078008C
:108F70002E40900080CF500003003100304180002F
:108F800090407800214798001E68EF000D003700E0
:108F90001EC8BF000080FB001E004000E1812000D1
:108FA000914078000181FB0061AC2000810041000C
:108FB00091407800014878001EC8BF000040E800DA
:108FC0001EE8B700E1812000914078002E4090001B
:108FD00080CF5000EEFF390003C4B30062AC200024
:108FE0008040EB0020C0B30019F607003041880034
:108FF0001EC8BF000080FA00000006000400FA004E
:10900000000F7800214798009EC0A9001FC8BF002C
:109010000004E00009003A009E0078000141880049
:10902000AE409000428220000149780010C0B30099
:1090300025E8B70010C0B3001FE8B7009EC0A80025
:109040000080FA00000006000600FA0020079800E1
:109050009EC0A9001FC8BF000004E000020032004B
:109060009EC0A8001F0037000040EB00004F7800B2
:10907000AE009000110798001E4FE8001E407800D7
:10908000E14F40000C0032001E00900010407800BC
:109090000080FB000000EA004F00DE000040780086
:1090A0009E0090008100E800110798000004E00095
:1090B000F1FF3A0001003700000000002E00900090
:1090C000004188009E4078004282200001497800DB
:1090D00010C0B30025E8B70010C0B3001FE8B70008
:1090E0009EC0A8000080FA00000006000600FA00FA
:1090F000200798009EC0A9001FC8BF000004E00020
:10910000020032009EC0A8001E0037000040EB00A5
:10911000004F7800AE009000110798001E4FE80045
:109120001E407800E14F40000C0032001E0090000D
:10913000104078000080FB000000EA004F00DE00D5
:10914000004078009E0090008100E8001107980020
:109150000004E000F1FF3A000100370000000000C9
:109160002E009000004188009E407800428220003E
:10917000014978002568EF0010C0B3001FE8B70070
:109180009EC0A8000080FA00000006000200FA005D
:109190009EC0A900404180000000E00008003200AD
:1091A00040418000900078000000280000806000AE
:1091B0000000E000020032009EC0A80062003700FC
:1091C0001FC8BF00E34F500001003A001F68EF00C6
:1091D0001FC8BF000004E00002003A009EC0A800C3
:1091E000590037001FC8BF00E24F500009003A0085
:1091F0008041EB000001EB0011C0B30020C0B300C0
:1092000093F507004041880030C0B3001FE8B70065
:109210004C0037001FC8BF00E14F500049003A0022
:10922000418220009140780000C4B30080CF5000FC
:109230000300360000C4B300004F7800030037007D
:109240004182200091407800014F780024C8BF007F
:109250001E40500024E8B70060A82000104188009C
:109260009E4078001147980025C8BF000004E00028
:109270001F003A000D0037001041800001418000BE
:109280009140780001487800104180000000E8001B
:1092900010418800004180000000E8000041880083
:1092A0001E4090000040E900104798001E409000CA
:1092B0000004E000F0FF3A00100037001041800089
:1092C0000141800091407800014878001041800001
:1092D0000000E80010418800004180000000E80024
:1092E000004188001E4090000040E90010479800AF
:1092F0001E4090000004E000F0FF3A0024C8BF00C8
:109300000004E00009003A0000C4B3009E40780069
:1093100080CF500003003A0020C0B3001FE8B70020
:109320000200370030C0B3001FE8B7009E4178004C
:1093300062A8200011C0B30020C0B30044F50700AC
:10934000404188009EC0A8000080FA00000006008E
:109350000800FA00881F780010079800220798007C
:10936000330798002E009000BE009000823E20003F
:109370000300200012EB07000002BE001E00900058
:109380008000EB000001BE000400BE000CEB0700F3
:10939000004478002E009000BE0090000268290072
:1093A0008309200006EB07000040780000405400CD
:1093B000004FE9001E80FB00A010880017E2A80003
:1093C0004F0478000080FA00000006000000FA0058
:1093D0001602A80000000000B010800061006000CC
:1093E0000000E000FCFF3A000080FA0000000600E8
:1093F0000000FA001622A80000000000B010800053
:10940000620060000000E000FCFF3A000080FA000B
:10941000000006000000FA001642A800000000004C
:10942000B0108000640060000000E000FCFF3A0023
:109430000080FA00000006000200FA00004F7800E9
:109440001E80FB009010880000000000C11080000A
:1094500000002400008060000000E000FBFF3A00F4
:10946000C01080004F00DE00004078000080FA004D
:10947000000006000400FA0020479800D3FF070010
:109480002E4090000004A100EBFF0700004F780081
:10949000E0FF07001E80FB000000E9004F00DE0037
:1094A000004078000080FA00000006000200FA0088
:1094B000004F780011479800C4FF07001E40780055
:1094C0000004A100DCFF07001E409000DAFF070047
:1094D000D0FF07000080FA00000006000400FA0038
:1094E000004F78001147980022479800B7FF070007
:1094F0001E4078000004A100CFFF07001E4090002E
:10950000CDFF07002E409000CBFF0700C1FF0700F2
:109510000080FA00000006000800FA0020479800CA
:109520002107980032079800A8FF07002E409000FE
:109530000004A100C0FF07000000EB00000F78004E
:10954000070037002E00900010407800BAFF070097
:109550002E0090000000E800200798001E0FE80091
:109560003E0090009E007800808F5000F5FF35008F
:10957000A8FF07000080FA00000006000400FA00BF
:109580002047980000000000B01080007F006000BD
:109590000000E000FCFF3A001662A8000000000096
:1095A000C0108000620060000000E000FCFF32009C
:1095B00080108000004F780000000000B010800094
:1095C0007F0060000000E000FCFF3A002E409000A9
:1095D000614060000080FB00610060004500DD002C
:1095E000B11080000150A10001007000B01088008F
:1095F0001682A80000000000B0108000700060001B
:109600000000E000FCFF3A001E4078000080FA00F5
:10961000000006000400FA00004F780011079800CF
:109620006AFF07001E4078000004A00082FF0700C8
:1096300010C0B300D1FF07009E0090008048780062
:1096400074FF07000080FA00000006000600FA0020
:10965000004F780011079800220798005BFF070071
:109660001E4078000004A00073FF07000040EB00DC
:10967000C2FF07009E0090008048780010C0B30031
:10968000BEFF0700AE0090008048780061FF070031
:109690000080FA00000006000800FA002047980049
:1096A000210798003207980048FF07002E409000DD
:1096B0000004A00060FF07000000EB00000F78002E
:1096C000110037003E0090000000E9009E0F50009E
:1096D000050032000040EB00A8FF0700AE0090003C
:1096E000804878000400370010C0B300A3FF0700D3
:1096F000AE009000804878002E0090000000E80046
:10970000200798001E0FE8003E0090009E007800A1
:10971000808F5000EBFF35003EFF07000080FA000D
:10972000000006000000FA0082C1B30011C0B300BF
:1097300000C9B30069FF07000080FA0000000600BE
:109740000400FA008040EB0000C9B30057FF070097
:109750008E80E800630047000101780080007800F7
:1097600000C9B300B9FF07003E4090000080FB0035
:109770004800DD00000F78002E4090000080FB00C4
:109780001E0040004580DE00000F7800F03F200002
:109790009E007800808F5000080034001E00EA0010
:1097A000CF80DE008CE907006022B80006002000B0
:1097B00007FC2B008CE90700070037001E0078002B
:1097C000CF80DE0084E907006022B8000600200098
:1097D00007FC230084E907000080FA00000006006F
:1097E0000200FA0011C0B30000C9B3002FFF070048
:1097F0008E00780000C9B30086FF07001E40780085
:109800000080FA00000006000400FA0021C0B30046
:1098100000C9B30025FF07008E80E8006300470001
:10982000010178008000780000C9B30087FF0700BD
:109830003E4090000080FB004800DD00000F7800F3
:109840002E4090000080FB001E0040004580DE009E
:10985000000F7800F03F20009E007800808F5000BD
:10986000080034001E00EA00CF80DE005AE907003D
:109870006022B8000600200007FC2B005AE9070010
:10988000070037001E007800CF80DE0052E9070095
:109890006022B8000600200007FC230052E9070000
:1098A0000080FA00000006000400FA0031C0B30096
:1098B00000C9B300FDFE07008E80E800630047008A
:1098C000010178008000780000C9B3005FFF070045
:1098D0003E4090000080FB004800DD00000F780053
:1098E0002E4090000080FB001E0040004580DE00FE
:1098F000000F7800F03F20009E007800808F50001D
:10990000080034001E00EA00CF80DE0032E90700C4
:109910006022B8000600200007FC2B0032E9070097
:10992000070037001E007800CF80DE002AE907001C
:109930006022B8000600200007FC23002AE9070087
:109940000080FA00000006000000FA00A6000700F0
:109950000CC8BF000004E000010032000DC8BF00C9
:109960000040FE00512480000002200000806000C2
:109970000000E00002003A0010C0B3004100070000
:10998000D200070010C0B3000080FA0000000600FB
:109990000000FA000CC8BF000004E00036003200EE
:1099A0000DC8BF000004E0003300320040248000F6
:1099B000620060000000E000010032008824A9007D
:1099C000750007000004200000248800000000004B
:1099D0000124800000042000008060000000E000FE
:1099E000FBFF32000004200000248800000000007B
:1099F0000124800000042000008060000000E000DE
:109A0000FBFF32000004200000248800000000005A
:109A10000124800000042000008060000000E000BD
:109A2000FBFF32009444A8000004200000248800BA
:109A3000000000000124800000042000008060007D
:109A40000000E000FBFF320000042000002488003A
:109A5000000000000124800000042000008060005D
:109A60000000E000FBFF32009444A900570007000B
:109A700010C0B300010037000040EB000080FA0086
:109A8000000006000400FA002047980040248000EF
:109A9000610060000000E0000B0032004024800004
:109AA000620060000000E00007003A001CC8BF0030
:109AB000E34F500004003600202480004300DE0005
:109AC00061406000320037002E4090000004E0004A
:109AD0001D0032008824A9008804A8002E00070079
:109AE0000040EB00004F7800090037000004200020
:109AF00000248800000000000124800000042000F1
:109B0000008060000000E000FBFF32001E4FE80014
:109B10001E407800E44F5000F4FF36000040EB0098
:109B20001047980020248000680060000000E000DA
:109B30000200320010C0B300104798002300070055
:109B40001E40900012003700402480006100600039
:109B50000000E00002003A0000C0EB000C003700FB
:109B600040248000620060000000E00002003A0033
:109B7000E0CFB300060037001CC8BF00E34F500021
:109B800002003E00D0CFB30001003700C0CFB300C9
:109B90000080FA00000006000000FA004668EF00AE
:109BA0001000FC00F1048000000420000080600030
:109BB0000000E0000200320010C0B30046E8B70029
:109BC0009EC0A9000080FA00000006000000FA0014
:109BD00046C8BF000004E000010032009EC0A8009B
:109BE0000080FA00000006000400FA001E00FC00DD
:109BF00011028000000E200000806000F04188000B
:109C000011028000000E2000010070001002880088
:109C100040092000100798000000EB00000F7800BA
:109C20000E0037001E009000900078001E007800A3
:109C300000014000C0BC2000000041000108780085
:109C40001E0090008000EB00010878001E009000CC
:109C50000080E800100798001E0FE8001E00780042
:109C6000E50F5000EFFF36006024800000428800BE
:109C70008C24EF0010248000104288008224EF0022
:109C8000700680004800DE00674060000080FB0036
:109C900020428800000120000024880000022000EB
:109CA000502488008EC0A9008284A800710680001C
:109CB000F08F2F000080600000A0A00070068800D8
:109CC0009EC0A8000080FA00000006000400FA0010
:109CD00040092000100798000000EB00000F7800FA
:109CE0000B0037001E00780080004000C0BC200040
:109CF00000804000900078001E009000010878006D
:109D00001E0090000080E800100798001E0FE80079
:109D10001E007800E50F5000F2FF36000042800080
:109D200060248800104280001024880020428000B7
:109D300000407800674060000080FB006700600022
:109D40004800DD0072068000F18F2F008100610065
:109D5000010070007006880011028000F0F12F00F1
:109D600080806000F041800001007000F0418800B8
:109D7000F0418000100288000080FA000000060018
:109D80000000FA000117800000F02F000080600042
:109D900000178800F002A900F022A900E822A9001B
:109DA000F402A900F422A900EC22A900005023002B
:109DB000C10020003E0307008040EB0080C3B300D9
:109DC000110007008040EB0080C0B3000E000700C8
:109DD0008040EB0010C0B3000B0007008040EB0098
:109DE00060C0B300080007008040EB00C0C0B300B3
:109DF0000500070000B82B00010020002C0307001D
:109E00000080FA00000006000400FA0020479800D5
:109E10003147980001178000F00F2000010070000A
:109E200000178800F422A800F402A900211780007E
:109E300000F02F000080600020178800EC22A800AE
:109E4000000000000000000000000000101780006B
:109E50004700DE0061406000004F7800EC22A9005E
:109E60001E4078000004E000F4FF3A000117800073
:109E700000F02F000080600000178800F422A90085
:109E80003E4090000080FB000000EA004F00DE0032
:109E9000004078000080FB0061006000A117800096
:109EA0000100A10001007000A017880021178000A8
:109EB00000F02F00808060002E4090000080FB00AA
:109EC0000100700020178800EC22A80000000000AC
:109ED0000000000000000000EC22A9000080FA0051
:109EE000000006000400FA00100798008F003700F9
:109EF0001E009000104F78001E00FB006101B900A9
:109F0000000520000100200002004000838048007E
:109F1000C204200003002000820F5000838F5800ED
:109F200075003E00006001007000370072003700CD
:109F300071003700700037006F003700680037008D
:109F40006D0037006C0037006B0037006A00370087
:109F50006900370068003700670037006600370087
:109F60006500370064003700630037006200370087
:109F700061003700600037005F0037005E00370087
:109F80005D0037005C0037005B0037005A00370087
:109F90005900370058003700570037005600370087
:109FA0005500370054003700530037005200370087
:109FB00051003700500037004F0037004E00370087
:109FC0004D0037004C0037004B0037004A00370087
:109FD0004900370048003700470037004600370087
:109FE0004500370038003700430037001B003700BA
:109FF00041003700400037003F0037003E00370087
:10A000003D0037003C0037003B00370016003700AA
:10A0100039003700380037003700370015003700A7
:10A0200035003700340037002A003700320037008F
:10A0300031003700120037002F0037001C003700B6
:10A040001E0037002C0037002B0037002A00370095
:10A050000E003700130037000F0037000040EB0000
:10A06000004F78002400370010C0B300004F780084
:10A070002100370020C0B300004F78001E003700D9
:10A0800030C0B300004F78001B00370040C0B30061
:10A09000004F78001800370050C0B300004F780020
:10A0A0001500370060C0B300004F78001200370081
:10A0B00070C0B300004F78000F003700F0CEB3003F
:10A0C000004F78000C00370080C0B300004F7800CC
:10A0D0000900370090C0B300004F78000600370039
:10A0E00040CEB300004F780003003700F0CDB3003E
:10A0F000004F7800000000001E407800EA4F50003A
:10A1000004003A008040EB0000CCB3003EFF0700A3
:10A11000030037001E40780011C0B3003AFF07006B
:10A120001E0090000000E800100798001E0090003C
:10A13000104078000004E0006DFF3A000080FA0053
:10A14000000006000200FA008040EB0000C4B300EB
:10A150002DFF07000000EB00000F7800060037001D
:10A16000C0112B001E0040001040780011C0B30049
:10A1700025FF07001E0FE800F00420009E00780075
:10A18000808F5000F6FF34008040EB0000C8B30021
:10A190001DFF07000080FA0000000600720B00009F
:10A1A0003400000000000000000800001E00000055
:10A1B00000000000000C0000300000000000000063
:10A1C000860A00009A000000000000001E0800003F
:10A1D0001200000000000000CC0B00000C0000008A
:10A1E000000000003E0800000A000000000000001F
:10A1F000A8090000DE000000000000003008000098
:10A200000E00000000000000200B000052000000C3
:10A210000200000030313200333435003637380068
:10A22000394142004344450046003000313233009A
:10A230003435360037383900616263006465660082
:10A2400000286E00756C6C00290000000100000001
:10A25000000A00000000640000000000E8030000A5
:10A26000001027000000A0008601000040420F00FF
:10A270000080960098000000E1F5050000CA9A00F1
:10A280003B000000A60B00002600000002000000BA
:10A29000D90B000000D90B000900000000020000EB
:10A2A000DB0B000000DB0B000E02010000000000D1
:10A2B0000000000000000000060202000000000094
:10A2C000A60B0000D80B00000600000000000000F4
:10A2D00048080000600100000200000000000000CB
:10A2E00000000000F03F000000000000000024001B
:10A2F0004000000000000000005940000000000085
:10A30000000040008F400000000000000088C300F3
:10A3100040000000000000006AF84000000000005B
:10A32000008084002E41000000000000D012630075
:10A330004100000000008400D797410000000000A9
:10A340000065CD00CD410000000020005FA00200AC
:10A3500042408C00B5781D00AF154400EA8CA00087
:10A3600039593E002946A5005CC3F10029633D0030
:10A37000489A64007EC50E001B514A0044F3C20097
:10A38000E4E4E900634C3D00C7DDD600BA2E770057
:10A390004E5FFB00F051EF00FC8A5000C7592900C6
:10A3A000090F6B009F527D00C3942500AD49B20098
:10A3B000545A6200D7D71800E77469009C750000F2
:10A3C000883CE400377E0000000000000000F00040
:10A3D0003F9A99009999990099B93F007B14AE0072
:10A3E00047E17A00843FFC00A9F1D2004D625000A1
:10A3F0003F2D43001CEBE200361A3F00F168E300FA
:10A4000088B5F800E43E8D00EDB5A000F7C6B000B9
:10A410003E48AF00BC9AF200D77A3E003A8C30003A
:10A42000E28E7900453E9500D626E8000B2E1100FD
:10A430003EBBBD00D7D9DF007CDB3D00234292004C
:10A440000CA19C00C73BA000C2EBFE004B48B4002F
:10A45000399C5700772726006CA137001FB8D4001D
:10A460004A7AEE008D352600A6ACAA0004B6790023
:10A47000339D35008F1DE9001566310023614D00C5
:10A4800017ACF800522F6F000E998400D94B400092
:10A490002D3005008EE42E00FF2B2B00ACF74E0074
:10A4A00015927E0068165900F3F8C2001F6EA500D1
:10A4B00001000000DE0B00000200000002000000AE
:10A4C00001000000000000000200FA00004F7800C8
:10A4D0001E80FB0040128800000000000012800077
:10A4E000610060000000E000FCFF320040128000CC
:10A4F000004078000080FA00000006000000FA002A
:10A50000D8E2A900DCE2A800A01320001012880005
:10A5100000002800001288000080FA0000000600F9
:10A520000200FA00DCE2A90050C0B300E6FF070019
:10A530000040EB00E4FF0700004F7800DCE2A800D9
:10A540001E4078000080FA00000006000000FA00BB
:10A55000DCE2A90060C0B300DBFF0700DCE2A8007A
:10A560000080FA00000006000000FA000000000071
:10A57000EBFF07000080FB006100600000407800F6
:10A580000004E000FAFF3A000080FA000000060034
:10A590000000FA00EDFF0700DCE2A90010C0B300E4
:10A5A000C9FF07000040EB00C7FF0700DCE2A8007E
:10A5B000EDFF07000080FA00000006000000FA002E
:10A5C000E2FF0700DCE2A90010C0B300BEFF0700F5
:10A5D000C0C8B300BCFF0700DCE2A800E2FF070030
:10A5E0000080FA00000006000400FA00100798003E
:10A5F000DCE2A90030C0B300B3FF07001E009000EA
:10A600004800DE0000407800AFFF07001E00900009
:10A6100000407800ACFF07000040EB00AAFF0700F5
:10A62000004F7800DCE2A8001E4078000080FA00AD
:10A63000000006000800FA00881F78001007980044
:10A640002107980062479800DCE2A90030C0B300FF
:10A650009DFF07001E0090004800DE0000407800CB
:10A6600099FF07001E0090000040780096FF070049
:10A670000000EB00000F7800070037001E00780094
:10A68000AE009000008440000040EB008EFF070009
:10A69000004C78001E0FE8006E4090000080FB0028
:10A6A0009E0F5000F5FF3C00DCE2A8004F0478004C
:10A6B0000080FA00000006000400FA00000F780095
:10A6C00021479800A1FF0700DCE2A90020C0B300E9
:10A6D0007DFF07001E0078004800DE000040780083
:10A6E00079FF07001E0078000040780076FF070021
:10A6F0002E40900074FF0700DCE2A8009AFF0700DC
:10A700000080FA00000006000800FA001007980018
:10A7100021079800624798000000EB00000F7800C6
:10A720008AFF0700DCE2A90020C0B30066FF070033
:10A730001E0090004800DE000040780062FF070025
:10A740001E009000004078005FFF07000000EB0053
:10A75000000F7800070037002E00900010407800AE
:10A76000AE0090008100E8002107980056FF070026
:10A770001E0FE8006E4090000080FB009E0F50000E
:10A78000F5FF3C00DCE2A80077FF07000080FA003C
:10A79000000006000800FA00000F7800110798007A
:10A7A0002207980033079800103A800000017800D3
:10A7B0000210A00060042000710520002374200016
:10A7C000804978008149780082497800540520004A
:10A7D000343B8800A40A2000343B880027A6A80048
:10A7E00027E6A90031318000003020000100700010
:10A7F000303188001E4078000080FB002031880046
:10A800001E4090000080FB00C800DD002E4090003C
:10A810000080FB0000804000203188003E40900016
:10A820000080FB00C800DD004E4090000080FB006F
:10A8300000804000203188005E4090000080FB00D6
:10A84000C800DD006E4090000080FB0000804000EA
:10A850002031880027E6A80027A6A9000080FA007A
:10A86000000006000E00FA000000000032318000F7
:10A8700001002100810061000100E000FBFF3A00BF
:10A880003231800001302000828070003131880038
:10A89000213180008140780061479800213180009B
:10A8A000010F78009E007800C808DE008140780023
:10A8B000714798009E00780081407800014F980011
:10A8C00021318000110798009E009000C808DE002A
:10A8D00081407800114F98009E00900081407800E0
:10A8E000214F98002131800021079800AE00900090
:10A8F000C808DE0081407800314F9800AE0090001B
:10A9000081407800414F9800E600470006000900AA
:10A91000315878007000B1000080FA000000060095
:10A920000A00FA00000F780011079800220798002B
:10A9300033079800044F980023E6A90011318000E6
:10A940000030200001007000103188001E407800A7
:10A950000080FB00003188001E4090000080FB005A
:10A96000C800DD002E4090000080FB000080400009
:10A97000003188003E4090000080FB00C800DD00F0
:10A980004E4090000080FB000080400000318800B5
:10A990005E4090000080FB00C800DD006E4090002B
:10A9A0000080FB0000804000003188000E489000CD
:10A9B0006F4060000080FB006F0060004A00DD0017
:10A9C00012318000F13F2C00810061000100700015
:10A9D0001031880023C6A80023E6A8000080FA00F2
:10A9E000000006000600FA00000F7800110798002A
:10A9F000220798001E00780021072000810F5000D8
:10AA00002100320021072000810F50000A003C0085
:10AA1000E20F50001E003200E20F500003003C0025
:10AA2000E10F5000130032001E003700E30F50000A
:10AA3000130032001B00370041072000810F500037
:10AA40000900320041072000810F5000120035003C
:10AA500051072000810F500011003A001000200023
:10AA6000210007000F003700200020001E00070013
:10AA70000C003700F4F807001CF707000900370046
:10AA80006CF80700070037000000000005003700E1
:10AA90000000000003003700000000000100370044
:10AAA0000000000010C0B3000080FA0000000600A3
:10AAB000F03FB1000180B10006003500EE0309004F
:10AAC00000000000403FB1000180B100FBFF3D00ED
:10AAD0001000B000203FB0000200350000800900E7
:10AAE00000000000000006000200FA00000F7800DD
:10AAF0001E007800E10F500002003A0092FB0700B0
:10AB000001003700000000000080FA00000006008D
:020000040001F9
:020000040002F8
:020000040003F7
:020000040004F6
:020000040005F5
:1057F000FFFF0000FFFF0000B62300007F3E000017
:00000001FF
